:1066E300011900000501013C0200000301FA040046
:1066F300FA0500030A0A5A0B001E0C00FA0D0003E8
:106703000E00040F0164100096120132130AFA14EA
:10671300010215000217010A1801FA1905321A01BC
:106723000A1B01FA1C05321FFFFF20FFFF23011E76
:106733002400642A00FA2B00FA2C50782D003D2EF9
:1067430000462F001E30006432507833000034328C
:10675300FA350164360164370150380A643C006439
:106763003E003C3F000140FFFF411450420A5A43A0
:106773000AC84405324500B44600FA470178480286
:10678300034C00FA4EFFFF500606510596520A329B
:10679300530B46540A9656010257054658000259B0
:1067A3000A465A32FA5B010A5C0A325E000A5F004B
:1067B300FE61FFFF64021C66000267FFFF6A0A3C7A
:1067C3006B00006C3296730000740000780132791C
:1067D30001327EFFFF81FFFF84FFFF8500AF86004C
:1067E300018700FA89010A8A00009900009D0A9630
:1067F3009E00019FFFFFA0FFFFFAFAFA00000501C8
:10680300013C0200000301FA0400FA0500030A0A2E
:106813005A0B001E0C00FA0D00030E00040F016456
:10682300100096120132130AFA1401021500001720
:10683300010A1801FA1905321A010A1B01FA1C058B
:10684300321FFFFF20FFFF23011E2400642A00FAEA
:106853002B00FA2C50782D003D2E00462F001E30C1
:1068630000643250783300003432FA350164360163
:1068730064370150380A643C00643E003C3F000129
:1068830040FFFF411450420A5A430AC844053245A7
:1068930000B44600FA47013C4802024C00FA4EFF9E
:1068A300FF500606510596520A32530B46540A9678
:1068B300560101570546580001590A465A32FA5BF8
:1068C300010A5C0A325E000A5F00FE61FFFF640397
:1068D3001C66000267FFFF6A0A3C6B00006C32967D
:1068E3007300007400007801327901327EFFFF816A
:1068F300FFFF84FFFF85FFFF86FFFF87FFFF8901FF
:10690300028A00009900009D0A969E00019FFFFFE6
:10691300A0FFFFFAFAFA0065006F00790083008D8B
:10692300009700A100AC00B600C000CA00D400DE8E
:1069330000E800F2005800600068007000780080F2
:1069430000880090009800A000A800B000B800C123
:1069530000C800D000D800DF00E600EE00F60041DA
:106963000047004D00530059005F0065006C007143
:106973000077007D00830089008F0095009B00A2B3
:1069830000A700AC00B200B900C000C500CA00D225
:0A69930000D500DD00E100E700EF91
:103A3900900054E0D3940440149007C5E0FEA3E03D
:103A4900FF9066E5126AD6E493F59980129007C54E
:103A5900E0FEA3E0FF9067FF126AD6E493F5999020
:103A690007C5E0FEA3E0FF9066E3E493FC740193CD
:103A7900FDEFB50507EEB50403754D009007C512B6
:103A89006ABD2275A71085F97385FA747E017F00D6
:103A9900E574126AAFE5732FFF50010E8E5A8F5BE2
:103AA900900017E0FCA3E0FDEF2DFDEE3CFC8C5CE3
:103AB9008D5D2275A71085F97385FA747E017F00E3
:103AC900E574126AAFE5732FFF50010E8E5A8F5BB2
:103AD900AC2CAD2DEF2DFDEE3CFC8C5C8D5D22E513
:103AE9005DF5FBE55CF5FCD29322E55DF5E9E55C66
:103AF900F5EAD29422E55DF5EBE55CF5ECD291228D
:103B0900E55DF5EDE55CF5EED29222E55DF5FDE5C5
:103B19005CF5FED28722E55DF5CEE55CF5CFD29066
:103B290022AE5AAF5B74068E048F05FF126A9F8C12
:103B39005C8D5DAE5AAF5B74068E048F05FF126A09
:103B4900CA8C5A8D5BE55B455A60137406C3955B55
:103B5900FFE4955AFE8E5A8F5B785C126B03E5730E
:103B6900A85CB80015D3955D4010E573C3955DFF5A
:103B7900E4955CFE8E5C8F5D8010E573243CC395F3
:103B89005DFFE4955CFE8E5C8F5DAE5CAF5D743B62
:103B99006F4E6006743C6F4E701AAE5CAF5D743B3D
:103BA9006F4E70057573018003757302755D3A7503
:103BB9005C00800375730022900095E0B40104C293
:103BC900108002D210900096E0B40104C211800264
:103BD900D2119000D3E075F0D2A4FFAEF0740A8E32
:103BE900048F05FF126A9F9007BBECF0A3EDF0A2CA
:103BF9000D401674038C068D07126AAF740112000A
:103C0900399007B9EEF0A3EFF07E017F00900091A3
:103C1900E0126AAF9000D4E08E048F05FF126A9F0C
:103C2900740AFF126A9F8D609000DDE075F0D2A4DE
:103C3900FFAEF0740A8E048F05FF126A9F9007BFCA
:103C4900ECF0A3EDF09000DFE060139000DFE0F509
:103C5900F0741684FF7E00EF9007CDF0800674643F
:103C69009007CDF09000D5E0900079F090011FE029
:103C7900900063F09000AEE0900065F09000D7E00E
:103C8900900066F0900083E0900067F0900109E0F1
:103C990090006CF090016DE090006DF090016EE085
:103CA90090006EF090016FE090006FF0A22AB3408F
:103CB9001690016DE0700C90016EE0700690016F36
:103CC900E060028002C22A74E3900078F09000BE9E
:103CD900E0B40B0874E3900078F0805A9000BEE0DD
:103CE900B419129000D4E090690412008CE4939006
:103CF9000078F080419000BEE0B41E129000D4E03C
:103D090090692212008CE493900078F0802890004A
:103D1900BEE0B428129000D4E090694C12008CE403
:103D290093900078F0800F9000BEE0B446089000B0
:103D3900B5E0900078F09000EEE0FE9000BCE06EF7
:103D4900600A9000BCE09000EEF0D22990007CE07F
:103D5900FE9000BBE0B5063390007EE0FE9000D9EE
:103D6900E0B5062790007DE0FE9000E7E0B5061B70
:103D7900900080E0FE90008EE0B5060F90007FE095
:103D8900FE9000C9E06E7003023F45900054E0C305
:103D990094055008740290010AF0801C9000C9E053
:103DA900640360069000E7E06008740790010AF078
:103DB9008006740A90010AF090008EE0B40106743E
:103DC900009000F4F090008EE0B4020674009000B8
:103DD900D9F090008EE0B4030674009000E6F090EC
:103DE90000BBE0601474189000A2F074009006CF34
:103DF900F074009006D0F0800C74009000A2F0746A
:103E0900189006CFF09000D9E0D3940140147419AA
:103E190090010CF074009006D3F074009006D4F071
:103E2900800C740090010CF074199006D3F0900086
:103E3900C9E0B403089000E7E064026002800674F8
:103E4900009000E7F09000E7E0B401089000C9E0B5
:103E590064036002801A741A90010DF074009000D6
:103E6900A3F074009006D7F074009006D8F0803360
:103E79009000BBE0B4021A741A9000A3F074009089
:103E8900010DF074009006D7F074009006D8F08008
:103E99001274009000A3F0740090010DF0741A9050
:103EA90006D7F09000C9E0B402069000E7E060028E
:103EB900801474049006E3F074059006E7F0740624
:103EC9009006EBF0802474009006E3F074009006ED
:103ED900E4F074009006E7F074009006E8F07400CE
:103EE9009006EBF074009006ECF0D2299000BBE04C
:103EF90090007CF09000E7E090007DF09000D9E020
:103F090090007EF09000C9E090007FF090008EE074
:103F1900900080F090008EE0900064F09000C9E07D
:103F2900900068F09000E7E0900069F09000BBE035
:103F390090006AF09000D9E090006BF09000F1E0F9
:103F4900B40117900023740FF0A374FFF0900025BB
:103F5900E4F0A3F074029000F1F09000F1E0B403F2
:103F690041900025E0FEA3E0FF900023E0FCA3E0E0
:103F7900FD126AFB7410126AAF7408120039EF90CF
:103F89000075F0EF700674FF900075F074009000F2
:103F9900F1F0900024E0900076F0900023E090008A
:103FA90077F0900082E0900043F0900043E0241401
:103FB900900044F0900043E02428900045F09000E0
:103FC90044E0D3943C400B900044E0C3943C9000FF
:103FD90044F0900045E0D3943C400B900045E0C389
:103FE900943C900045F0900049E4F0900043E0646F
:103FF9003B6007900043E0B43C20900043E0B43BB1
:10400900067402900049F0900043E0B43C06900029
:10401900497401F09000437401F090004AE4F09073
:104029000044E0643B6007900044E0B43C20900009
:1040390044E0B43B06740290004AF0900044E0B4B6
:104049003C0690004A7401F09000447401F090001D
:104059004BE4F0900045E0643B6007900045E0B414
:104069003C20900045E0B43B06740290004BF09070
:104079000045E0B43C0690004B7401F09000457493
:1040890001F0900082E0FE9000E5E02E90004DF0F6
:104099009000C0E0B4016390004DE0641E60079099
:1040A900004DE0B43C0690004DE004F090004DE076
:1040B900641D600790004DE0B43B0690004DE0148C
:1040C900F090004DE0D3943C400B90004DE0C39438
:1040D9003C90004DF090004DE0D3941E400D9000AF
:1040E9004DE0C3941E90004EF0800A90004DE024EC
:1040F9001E90004EF075511E807990004DE06414B9
:10410900600F90004DE06428600790004DE0B43CDA
:104119000690004DE004F090004DE06413600F90AC
:10412900004DE06427600790004DE0B43B06900025
:104139004DE014F090004DE0D3943C400B90004DBD
:10414900E0C3943C90004DF090004DE0D3941440AE
:104159000B90004DE0C3941490004DF090004DE099
:10416900D39414400B90004DE0C3941490004DF08B
:104179007551149000C8E0900046F0900046E07533
:10418900F01484AFF07E00EF4E7006900046E00414
:10419900F0900046E00475F01484AFF07E00EF4E15
:1041A9007006900046E014F0900046E0B47906905D
:1041B90000467401F0900046E0D3943C400F900013
:1041C90046E0C3943C900046F0D2238002C223907B
:1041D9000046E02414900047F0900046E02428901F
:1041E9000048F0900047E0D3943C400B900047E032
:1041F900C3943C900047F0900048E0D3943C400BB6
:10420900900048E0C3943C900048F022C293C294C5
:10421900C291C292C287C290E5B554EFF5B5E5B532
:1042290054DFF5B5C296C295C2A0C297C2A2C2A177
:10423900E5B554BFF5B5E5B5547FF5B5E5B554FB1E
:10424900F5B5C212755E469000CBE07005756D023A
:104259008003756D0375550075540090000C74FF4B
:10426900F0A374DCF0C218C21AC21C74C8900037DB
:10427900F074C890003BF074C890003FF07553008B
:10428900755200C20D754600E56FB40903756F00DC
:10429900756300900019E4F0A3F0757010C215C29F
:1042A90016C2179007BBE0FEA3E0FF7403126AAFC2
:1042B90074011200399007B9EEF0A3EFF0C202754C
:1042C9005700755600900010E4F0A3F0C22B755901
:1042D9000075580090008DE075F032A4FDACF090A7
:1042E9000021ECF0A3EDF0C23BA22FB39205A2305E
:1042F900B39206A231B39207A232B39208A233B3A2
:104309009209A234B3920AA235B3920BA236B392A0
:104319000C2275A71085F97385FA747E017F00E573
:1043290074126AAFE5732FFF50010E8E5A8F5BAC82
:104339005CAD5DEF2DFDEE3CFC8C5C8D5D123AE8C9
:10434900123AF3123AFE9000C9E0B40309123B098C
:10435900123B14123B1F75A7002285F97385FA7465
:104369007E017F00E574126AAFE5732FFF50010EDD
:104379008E5A8F5B7E017F76900106E0126AAFACA0
:104389005AAD5BED2FFFEC3EFE8E5C8F5DE55DF572
:10439900EDE55CF5EE900079E4F07412900050F0D0
:1043A9002285F97385FA747E017F00E574126AAF7C
:1043B900E5732FFF50010E8E5A8F5B9007BBE0FC0F
:1043C900A3E0FDEF2DFDEE3CFC8C5C8D5DE55DF51C
:1043D900FDE55CF5FE22056422A2DBB340089000EE
:1043E900D5E0900079F0A2DCB34006C296C295C22E
:1043F900A075D8402285A77275A7109000C9E064FE
:104409000360079000E7E0B4022CA2D8B34002C2CF
:1044190093A2D9B34002C294A2DAB34002C291A2D4
:10442900DBB34002C292A2DCB34002C287A2DDB371
:104439004002C290802DA2D8B3400AC2939000E7EF
:10444900E06002C292A2D9B3400AC2949000E7E0A8
:104459006002C287A2DAB3400AC2919000E7E06025
:1044690002C29075D8408572A722900047E49364F0
:1044790006600280FE74C89007C1F8E4F0E8A3F072
:1044890075B50075840175A70075FFA090004CE40F
:10449900F075C91075A70F75A1C775A70075D90063
:1044A90075CE0C75A70F75F1FE75F2FF75F30775DB
:1044B900F47875A4BA75A5FF75A60775AE0075AF32
:1044C900FF75D48175D5FF75D6FF75D7FF75A70020
:1044D90075A20175A14775F80975D80075D90475D4
:1044E900DD0975DE0975D84075A71075D80075D92D
:1044F9000475DA0975DB0975DC0975DD0975DE09ED
:1045090075DF0975D84075A70075E60875E7107558
:10451900BC0175BE0475BD6C75BE0775BDA075BEC1
:104529000875BD0175BC0075BB1875BC2075BA0846
:1045390075E88075D11375A70F75E10575E20075EA
:10454900C740124215759700759780740A126A8FD1
:104559007597C0E5975420700280F8758F0275A78A
:1045690000D2AF75980075A90C75A70F75AB437587
:10457900ADFB75AC1E75A71075C91875CA0075CB4A
:104589000075C80475A700758912758E04758C00AD
:10459900758A00C2A9D28C758D00758B00D2ABD2F9
:1045A9008E75EF0675D944C29974C8F50975080066
:1045B9001200E975B5001204E974639007C1F8E4C3
:1045C900F0E8A3F012037574C89007C1F8E4F0E8A5
:1045D900A3F07464F5097508001200E9900064E01D
:1045E90090008EF090008EE0D39403400C740090FC
:1045F900008EF07400900064F0C22090008EE0906C
:1046090062F4F82828738028A2B44002D2208020BE
:1046190075A70F75F30F75A700A2A34002D22080DA
:104629000F75A70F75F31775A700A2A44002D22032
:0C62F40002460F02461102461902462A1B
:10463900A220B3405F757308E573D3940E5020E54B
:10464900739007C1F8E4F0E8A3F01202447464F52A
:10465900097508001200E97873740126F650D974B7
:10466900029000CAF0900064E090008EF090008EF5
:10467900E0906300F8282873801674009000F4F025
:10468900800E74009000D9F0800674009000E6F066
:0C63000002468102468302468B0246934F
:10469900D21F805D757301E573D394075020E573CC
:1046A9009007C1F8E4F0E8A3F01202447464F50934
:1046B9007508001200E97873740126F650D974015F
:1046C9009000CAF0900064E090008EF090008EE0B7
:1046D90090630CF8282873801674009000F4F08019
:0F46E9000E74009000D9F0800674009000E6F087
:0C630C000246E00246E20246EA0246F2C7
:1046F800C21F900063E090011FF0900064E09000FA
:104708008EF0900065E09000AEF0900066E09000BA
:10471800D7F0900067E0900083F0900068E0900088
:10472800C9F0900069E09000E7F090006AE090001E
:10473800BBF090006BE09000D9F090006CE0900125
:1047480009F090006DE090016DF090006EE090012E
:104758006EF090006FE090016FF090016DE0700CCA
:1047680090016EE0700690016FE060028004C22A3A
:104778008002D22A9000D4E07006740A9000D4F027
:104788009000B5E0700674E39000B5F09000BBE0CF
:104798000490007CF09000BCE09000EEF0123BC169
:1047A800E5B54401F5B57406900052F07401900027
:1047B80053F07403900055F07405900056F0741E81
:1047C800900057F07405900058F0900054E0B4043D
:1047D800067404900058F07401900059F074009029
:1047E800005EF07400900061F074FF900062F07455
:1047F80036900158F07430900159F0742D90015A98
:10480800F0743290015BF0742090015CF074369083
:10481800015DF0744390015EF0747990015FF0746B
:104828006C900160F07420900161F0742090016236
:10483800F07420900163F07420900164F07420906B
:104848000165F07420900166F09000F0E09000752A
:10485800F09000A7E0900076F09000A8E090007734
:10486800F0A2B6B3920EA2B3B3920FA2A4B392264B
:10487800A2B4B39227A2A3B39228900071E4F07572
:104888006F00743A900781F074FD900782F09000F1
:1048980072E4F09007BBE0FEA3E0FF7403126AAF76
:1048A80074011200399007B9EEF0A3EFF0756E01AC
:1048B800900050E4F0C225756300C213D214C202FE
:1048C800757100C22DD203C22ED204C22FD205C2E6
:1048D80030D206C231D207C232D208C233D209C29C
:1048E80034D20AC235D20BC236D20CC221C222C27D
:1048F80023C224C22912009E755F00756B00756182
:104908000075653275660075670075680075690021
:10491800756A00900019E4F0A3F0756C00D2B2D269
:10492800A4D2B0D2B1D2A3D2A7D2A6D2A5D2B790E0
:10493800008DE0D394FA400674FA90008DF07E0161
:104948007F00900077E0126AAF900076E02FFF506A
:10495800010E900023EEF0A3EFF0EFD394FFEE9456
:104968000F4007900023E4F0A3F0900075E0700674
:1049780074FF900075F09000CAE0D394024006746A
:10498800019000CAF09000CBE07005756D028003BD
:10499800756D039000CCE0D394014006740090003C
:1049A800CCF09000D2E0C3940A5006740A9000D26A
:1049B800F09000DCE0700674019000DCF09000DC00
:1049C800E0B4FF0674FE9000DCF09000E3E0D394BE
:1049D800FE400674FE9000E3F0900109E0D39402D3
:1049E80040067401900109F090011FE0D394014042
:1049F80006740190011FF074019000E9F0740190B1
:104A080000EAF074009000F1F07400900111F07465
:104A1800299006C7F0742A9006CBF0741B9006DB29
:104A2800F0741C9006DFF0D29C9000BCE0D3940494
:104A3800400674049000BCF0E570D39410400375F0
:104A480070109006C8E0D3940C400674009006C815
:104A5800F09006CCE0D3940C400674009006CCF09D
:104A68009006D0E0D3940C400674009006D0F090E5
:104A780006D4E0D3940C400674009006D4F0900657
:104A8800D8E0D3940C400674009006D8F09006DC69
:104A9800E0D3940C400674009006DCF09006E0E049
:104AA800D3940C400674009006E0F09006E4E0D33E
:104AB800940C400674009006E4F09006E8E0D39465
:104AC8000C400674009006E8F09006ECE0D3940CD5
:104AD800400674009006ECF0D2EC75CF01A298B3B2
:104AE8004005C298120646E54D6006A299B3B34048
:104AF800028005C299120C57E54E64016005E54E27
:104B0800B4040280D5C28E7E107F00E564126AAFBD
:104B1800E58D75F010A4FDACF0EF2DFDEE3CFCE545
:104B28008B75F01084FF7E00ED2FFFEC3EFE8E5457
:104B38008F55D28E9000AEE060099000AEE0C3942D
:104B48003D4002805690001B126ABD90001BE0FE9B
:104B5800A3E0FF90001DE0FCA3E0FDEFB5053CEEEF
:104B6800B50438B21EA20DB34013A21EB34008E527
:104B7800B54404F5B58006E5B554FBF5B590001DC0
:104B8800E0FEA3E0FF90001FE0FCA3E0FDEF2DFD99
:104B9800EE3CFC90001DECF0A3EDF09000BBE06053
:104BA800099000BBE0C394034002806F122D96A2C7
:104BB8000DB35009900071E0C3942B400280069019
:104BC80000A5E0F545E54575F005A4FFAEF09007B2
:104BD800C3EEF0A3EFF0900092E0C395614007E5C3
:104BE8005FC3956050079007C3E4F0A3F0AE2EAF03
:104BF8002F9007C3E0FCA3E0FDEFD39DEE9C40049B
:104C0800C297800B900071E0C394415002D29790F4
:104C180000BBE0B40205A297B392A19000BBE0B438
:104C2800031C122EB1AE2EAF2F9007C3E0FCA3E0F9
:104C3800FDEFD39DEE9C4004D2978002C29790006E
:104C480096E06009A2B3300F01B3B340028039A2E5
:104C5800B3300F01B34031A2B3301101B3401C90FF
:104C680000C9E0B40306A221B3B34002800674046D
:104C7800900050F0D221A211B3920FA211B330B319
:104C880001B34004A211920FA2B6300E01B3500333
:104C9800025325A2B6300E01B35003025325A2B623
:104CA800301001B35003025167756E009000AEE0FA
:104CB800B43D13A210B34008E5B554FBF5B5800622
:104CC800E5B54404F5B5055EA212B3B35013AE546E
:104CD800AF5590000CE0FCA3E0FDEDC39FEC9E40B7
:104CE80003024E37E56DB4032EA22BB34022E55ED6
:104CF800B43B03756D01E55EC3943B5006900050CC
:104D08007401F0E55ED3943B40067402900050F0C5
:104D1800755E01D22B805CE56DB40206756D017578
:104D28005E3BE55EB43B05755E018047900050E050
:104D38007032E55EC3943B50069000507401F0E574
:104D48005ED3943B40067402900050F0E55EC39435
:104D58003B5002D225E55ED3943B4002D225C29651
:104D6800C295C2A09000CBE0B401051242158003A1
:104D7800755E01AE56AF57AC54AD55EF2DFDEE3C08
:104D8800FC74028C068D071200398E568F579000DE
:104D9800AEE060099000AEE0C3943D4002804390CD
:104DA800001BE0FEA3E0FF9000AEE08E048F05FF3D
:104DB800126A9F74018C068D0712003990001FEE4D
:104DC800F0A3EFF090001FE0F8A3E090001DC8F0FA
:104DD800A3C8F090001BE4F0A3F0C21EE5B554FB95
:104DE800F5B5A2B4B34002C227A2A4B34002C226BA
:104DF800A2A3B34002C228A225B34002C225A22121
:104E0800B34006A22392228002B222900096E0606C
:104E180012E56D700EA221B35009A222302301B30E
:104E2800B3400280067405900050F0C221803AAE6B
:104E380056AF57AC54AD55EF2DFDEE3CFC74018CCC
:104E4800068D071200398E568F57E56DC3940250B0
:104E58000DAC54AD5574B8C39D740B9C40028009C9
:104E68001242157406900050F0E55EB43B127403CC
:104E7800900050F0D2259000CBE0B4010312421507
:104E8800AE58AF59AC54AD55EF2DFDEE3CFC8C58E7
:104E98008D59AE54AF55EFD39DEE9C401190001341
:104EA800E0FAA3E0FBEBC394E8EA9403400280062F
:104EB800900013126ABD900010E0FEA3E0FFAC540E
:104EC800AD55EF2DFDEE3CFC900010ECF0A3EDF09D
:104ED8009000CBE0B40118AE54AF557405126AAF18
:104EE800740112003990000CEEF0A3EFF08011AEBF
:104EF80054AF557402126AAF90000CEEF0A3EFF0B5
:104F0800C28E758D00758B007564007555017554DA
:104F180000D28EE55E240E75F00F84AFF07E00EFB0
:104F28004E7075900010E0F8A3E090000EC8F0A352
:104F3800C8F090000EE0FEA3E0FFEF4E600B7C7916
:104F48007DC212699D8E528F53900010E4F0A3F039
:104F5800AE52AF537428BE00039F5010E5632FFF75
:104F680050010E74011200398E528F53855363908D
:104F780000D2E0A852B8000DD395534008E55390ED
:104F8800004FF080099000D2E01490004FF0E56DDA
:104F980060067553007552009000C9E0B40308908C
:104FA8000046E0655E6002800BA222B34004D22472
:104FB8008002B224E55E640B6005E55EB4290990C1
:104FC80000BBE060031223D29000C0E0B40114904B
:104FD800004DE0655E600790004EE0B55E03756FBA
:104FE80000801E90004DE0655E601390004DE02447
:104FF80014655E600990004DE02428B55E03756F66
:1050080000A213B35006A212B3B340030250BC90DF
:105018000087E0B40173900109E0B40214120E266F
:1050280090007AE075F0BEA4FFAEF08E5C8F5D80D4
:1050380056E56775F00A84FF7E00900581126AD6EE
:10504800E0F55B755A00AE5AAF5B9000ACE0126AAF
:10505800AF74648E048F05FF126A9F8C5C8D5DE5CA
:105068005D900012F0AE5AAF5B900085E0126AAF17
:1050780074648E048F05FF126A9F74BE8C068D07B8
:10508800126AAF8E5C8F5D8017900085E075F0BE68
:10509800A4FFAEF08E5C8F5D9000ACE0900012F043
:1050A800E561C394CC5006E55D455C70028003124F
:1050B800431BD213E56DB40106E55E6411600280FE
:1050C800097570019000517401F0E56D600302519B
:1050D800629000CEE0600D900079E0A852B800061A
:1050E8009553400280409000CEE0B4021F900043E8
:1050F800E0655E600F900044E0655E6007900045E3
:10510800E0B55E03757003756C00800CC200756CA9
:1051180000900019E4F0A3F0900079E060067409AB
:10512800900050F08034900043E0B55E0B7570013C
:105138009000517401F08022900044E0B55E0B7538
:1051480070017402900051F08010900045E0B55E47
:10515800097570017403900051F0A210B3920EA269
:1051680010B330B601B35003025325756E01900099
:10517800AEE0B43D13A210B34008E5B54404F5B55C
:105188008006E5B554FBF5B5E5B54401F5B5742BD6
:10519800900071F0A210920EE55ED3944A4014D2AA
:1051A80012E55ED39485400B7404900050F0D2252C
:1051B800755E469000D6E0B40107E56AC3941440D2
:1051C8000280091242157413900050F0A22D30038A
:1051D80001B35017A22DB34008E5B54408F5B580D2
:1051E80006E5B554F7F5B5A22D9203A22E300401B9
:1051F800B35017A22EB34008E5B54402F5B58006B2
:10520800E5B554FDF5B5A22E9204A22F300501B3E1
:10521800500FA22FB34004D2978002C297A22F92B8
:1052280005A230300601B3500FA230B34004D2A219
:105238008002C2A2A2309206A231300701B3500FF9
:10524800A231B34004D2A18002C2A1A2319207A226
:1052580032300801B35017A232B34008E5B54440D4
:10526800F5B58006E5B554BFF5B5A2329208A2336C
:10527800300901B35017A233B34008E5B54480F5AF
:10528800B58006E5B5547FF5B5A2339209A234304E
:105298000A01B3500FA234B34004D2928002C292E2
:1052A800A234920AA235300B01B3500FA235B34095
:1052B80004D2878002C287A235920BA236300C0135
:1052C800B3500FA236B34004D2908002C290A236E7
:1052D800920CE56AC394415009740E900050F01284
:1052E8004215900058E0FE900054E004C39E400927
:1052F800900054E0D39408400974FB900050F012D9
:10530800421590005DE0601590005DE0FE9000574A
:10531800E06E600974FE900050F0124215A225B3A9
:105328004006C296C295C2A0900106E0600CAE523B
:10533800AF537414BE00059F4002804890008EE071
:10534800906318F8282873803BA2B4B35005A227AD
:10535800B340028005124363D2278028A2A3B3502A
:1053680005A228B340028005124363D2288015A203
:10537800A4B35005A226B340028005124363D22687
:04538800800280001F
:1063180002534F02535102536402537702538A02C5
:02632800538C94
:10538C00A215B3B35008900046E0655E600302546A
:10539C0021A201B35006A200B3B340028071900069
:1053AC00C9E0B40343123A8CA20DB34021A224B33A
:1053BC004005123AE88003123B099000E7E0B40183
:1053CC000BA202B34004D2A18002C2A18018123AEF
:1053DC00E8123B099000E7E0B4010BA202B34004D1
:1053EC00D2A18002C2A180249000E7E0C3940250B5
:1053FC000F123A8C123AE8A202B34002D292800CFD
:10540C00123A8C123AE8123ABC123B0975A700C248
:10541C0015D216D217A216B3B35008900047E06508
:10542C005E60030254B6A201B35006A200B3B340AF
:10543C000280719000C9E0B40343123A8CA20DB300
:10544C004021A224B34005123AF38003123B14907E
:10545C0000E7E0B4010BA202B34004D2A18002C267
:10546C00A18018123AF3123B149000E7E0B4010B40
:10547C00A202B34004D2A18002C2A180249000E712
:10548C00E0C39402500F123A8C123AF3A202B340CA
:10549C0002D287800C123A8C123AF3123ABC123BAD
:1054AC001475A700D215C216D217A217B3B35008A1
:1054BC00900048E0655E600302554BA201B35006B4
:1054CC00A200B3B3400280719000C9E0B403431250
:1054DC003A8CA20DB34021A224B34005123AFE80AF
:1054EC0003123B1F9000E7E0B4010BA202B340048F
:1054FC00D2A18002C2A18018123AFE123B1F90006A
:10550C00E7E0B4010BA202B34004D2A18002C2A115
:10551C0080249000E7E0C39402500F123A8C123AA8
:10552C00FEA202B34002D290800C123A8C123AFEC8
:10553C00123ABC123B1F75A700D215D216C217E542
:0F554C007090632AF8282873025A979000BCE0E9
:06632A0002555402555714
:10555B0090635DF8282873121EAE8012121EAE8067
:0E556B000D121F388008121FE48003121FE487
:0F635D0002556202556702556C02557102557662
:10557900757002025A97122110122227A23BB340DA
:10558900229000B0E0F56C900081E0256CFE90005F
:105599004FE075F01E84FC7F00EE2CF536741090F8
:1055A9000050F09007B9E0FEA3E0FF740A126AAF59
:1055B90090000EE0FCA3E0FD74098F02FF126A9FC0
:1055C9008D078C038E048A058B0612699D9007BD91
:1055D900EEF0A3EFF09000D7E0B401087450BE00DC
:1055E900059F4002800D74509007BDF8E4F0E8A3D0
:1055F900F0801B9007BDE0FEA3E0FF74F0BE00033E
:105609009F500B74F09007BDF8E4F0E8A3F0E5367D
:1056190070037536019007BDE0FEA3E0FFE5362F64
:10562900FF50010E9007BDEEF0A3EFF075700390E7
:035639000051E03D
:0363300002557F94
:10563C0090636CF82828738019A23C400375700A9B
:10564C008010A23C400375700B8007A23C40037590
:02565C00700CD0
:0C636C0002564302564502564E02565798
:10565E00025A979006C8E060031224EA900107E010
:10566E00B40114900108E0A852B8000495535007F5
:10567E00E55FC39560400280097415900050F002FA
:10568E0057119000BCE0D39402403F900090E0246C
:10569E0003A852B8000495535009900092E0D39598
:1056AE006150028008D2017408900050F090009072
:1056BE00E0A852B80005D39553500B900092E02409
:1056CE0003C395615002C2018039900090E024031B
:1056DE00A852B8000495535007E55FC39560400289
:1056EE008008D2017408900050F0900090E0A8520B
:1056FE00B80005D395535009E560240FC3955F504C
:10570E0002C2019000D6E07007E56AC3941440020D
:10571E008002D201A2014005757004800A757010D6
:10572E00900019E4F0A3F0A20DB34029E56775F0DF
:10573E000A84FF7E00900581126AD6E0C3946950F8
:10574E0005122407800F9007BBE0F8A3E09007B97D
:0C575E00C8F0A3C8F0025A979000BCE00D
:06633300025661025766EC
:10576A00906378F8282873120F108012120F108095
:0E577A000D1210BE8008121170800312117003
:0F63780002577102577602577B025780025785F2
:105788009006CCE060031225C6757005025A971280
:1057980012B07570069006D0E060031226B6900627
:1057A800D4E06003122792025A97900012E0600634
:1057B800A20DB3B34002801D900012E02529FFAE70
:1057C8002850010E8E288F29E55ED3941450069038
:1057D8000012E014F01214F67570079006D8E06015
:1057E8000312286E9006DCE0600312294A025A97D9
:1057F800900109E0B40203120E9E1218F5757008A4
:105808009006E0E06003122A269006E4E0600312A6
:105818002B02025A97121CB1A215B35005A216B357
:1058280040028006D215D216D2177570109006E87D
:10583800E06003122BDE9006ECE06003122CBA0243
:105848005A97025A97900039E0C394465008C29676
:105858007446900039F0900049E0B4011DE5362403
:1058680006F5369007BDE0FEA3E0FF74062FFF5053
:10587800010E9007BDEEF0A3EFF0900049E0B402EE
:105888001DE536240CF5369007BDE0FEA3E0FF7455
:105898000C2FFF50010E9007BDEEF0A3EFF08536F8
:1058A8005B755A00900043E0F573123B2AE55D9062
:1058B8000039F0900006E55AF0A3E55BF0E5739037
:1058C800003AF0C2199007BDE0F55AA3E0F55B90E5
:1058D8000043E0F573123B2AE55D900037F0900035
:1058E80000E55AF0A3E55BF0E573900038F0C218C4
:1058F800E56DB4010575700B8003757003025A9746
:1059080090003DE0C3944650139000D7E0B40104E2
:10591800C2968002C295744690003DF090004AE01D
:10592800B4011DE5362406F5369007BDE0FEA3E078
:10593800FF74062FFF50010E9007BDEEF0A3EFF0A5
:1059480090004AE0B4021DE536240CF5369007BDF8
:10595800E0FEA3E0FF740C2FFF50010E9007BDEE90
:10596800F0A3EFF085365B755A00900044E0F573BC
:10597800123B2AE55D90003DF0900008E55AF0A33F
:10598800E55BF0E57390003EF0C21B9007BDE0F5C3
:105998005AA3E0F55B900044E0F573123B2AE55DFD
:1059A80090003BF0900002E55AF0A3E55BF0E57348
:1059B80090003CF0C21AE56DB4010575700C8003C7
:1059C800757003025A97900041E0C39446501390B3
:1059D80000D7E0B40104C2968002C2A074469000C9
:1059E80041F090004BE0B4011DE5362406F53690F1
:1059F80007BDE0FEA3E0FF74062FFF50010E9007DD
:105A0800BDEEF0A3EFF090004BE0B4021DE53624A4
:105A18000CF5369007BDE0FEA3E0FF740C2FFF5095
:105A2800010E9007BDEEF0A3EFF085365B755A00C6
:105A3800900045E0F573123B2AE55D900041F09037
:105A4800000AE55AF0A3E55BF0E573900042F0C266
:105A58001D9007BDE0F55AA3E0F55B900045E0F521
:105A680073123B2AE55D90003FF0900004E55AF080
:105A7800A3E55BF0E573900040F0C21CE56DB4014E
:0F5A880003756D00757003800680048002800036
:106339000257970257B20257F802581D02584A02EB
:10634900584D0259080259CE025A91025A93025ADB
:0463590095025A97B8
:105A9700900037E0B55E028003025B39A2184072BE
:105AA700900000E0FEA3E0FFEF4E6021AE56AF5737
:105AB700900000E0FCA3E0FD12000374068E048F43
:105AC70005FF126A9F900000ECF0A3EDF0900038FC
:105AD700E0601A900000E0FEA3E0FFAC56AD57EF80
:105AE7002DFDEE3CFC900000ECF0A3EDF0900038AB
:105AF700E0D39401401A900000E0FEA3E0FFAC560B
:105B0700AD57EF2DFDEE3CFC900000ECF0A3EDF05F
:105B1700D218AE54AF55900000E0FCA3E0FDEFC3F0
:105B27009DEE9C400D1243AAD296C21874C89000ED
:105B370037F0A218B3B35007900037E0B55E028084
:105B47000D1243AAD29674C8900037F0C21890007D
:105B570039E0B55E028003025BF4A219407290003F
:105B670006E0FEA3E0FFEF4E6021AE56AF57900070
:105B770006E0FCA3E0FD12000374068E048F05FF08
:105B8700126A9F900006ECF0A3EDF090003AE060F7
:105B97001A900006E0FEA3E0FFAC56AD57EF2DFDCF
:105BA700EE3CFC900006ECF0A3EDF090003AE0D359
:105BB7009401401A900006E0FEA3E0FFAC56AD57F3
:105BC700EF2DFDEE3CFC900006ECF0A3EDF0D219B2
:105BD700AE54AF55900006E0FCA3E0FDEFC39DEE89
:105BE7009C400AC2967446900039F0C219A219B3B4
:105BF700B35007900039E0B55E02800AC29674463A
:105C0700900039F0C21990003BE0B55E02800302B4
:105C17005CBAA21A4072900002E0FEA3E0FFEF4ECA
:105C27006021AE56AF57900002E0FCA3E0FD1200E2
:105C37000374068E048F05FF126A9F900002ECF032
:105C4700A3EDF090003CE0601A900002E0FEA3E0B4
:105C5700FFAC56AD57EF2DFDEE3CFC900002ECF08B
:105C6700A3EDF090003CE0D39401401A900002E0CD
:105C7700FEA3E0FFAC56AD57EF2DFDEE3CFC9000C8
:105C870002ECF0A3EDF0D21AAE54AF55900002E04B
:105C9700FCA3E0FDEFC39DEE9C40181243AA9000C1
:105CA700D7E0B40104D2968002D295C21A74C89084
:105CB700003BF0A21AB3B3500790003BE0B55E0279
:105CC70080181243AA9000D7E0B40104D29680024C
:105CD700D29574C890003BF0C21A90003DE0B55EC3
:105CE700028003025D8BA21B4072900008E0FEA3B6
:105CF700E0FFEF4E6021AE56AF57900008E0FCA3DF
:105D0700E0FD12000374068E048F05FF126A9F9050
:105D17000008ECF0A3EDF090003EE0601A90000858
:105D2700E0FEA3E0FFAC56AD57EF2DFDEE3CFC9037
:105D37000008ECF0A3EDF090003EE0D39401401A88
:105D4700900008E0FEA3E0FFAC56AD57EF2DFDEE47
:105D57003CFC900008ECF0A3EDF0D21BAE54AF551D
:105D6700900008E0FCA3E0FDEFC39DEE9C4015907A
:105D770000D7E0B40104C2968002C2957446900031
:105D87003DF0C21BA21BB3B3500790003DE0B55EC8
:105D97000280159000D7E0B40104C2968002C29534
:105DA700744690003DF0C21B90003FE0B55E028054
:105DB70003025E5CA21C4072900004E0FEA3E0FFB9
:105DC700EF4E6021AE56AF57900004E0FCA3E0FD14
:105DD70012000374068E048F05FF126A9F90000459
:105DE700ECF0A3EDF0900040E0601A900004E0FEB4
:105DF700A3E0FFAC56AD57EF2DFDEE3CFC90000441
:105E0700ECF0A3EDF0900040E0D39401401A90002D
:105E170004E0FEA3E0FFAC56AD57EF2DFDEE3CFCD2
:105E2700900004ECF0A3EDF0D21CAE54AF559000F7
:105E370004E0FCA3E0FDEFC39DEE9C40181243AACB
:105E47009000D7E0B40104D2968002D2A0C21C749D
:105E5700C890003FF0A21CB3B3500790003FE0B5D5
:105E67005E0280181243AA9000D7E0B40104D296CC
:105E77008002D2A074C890003FF0C21C900041E09D
:105E8700B55E028003025F2DA21D407290000AE0FA
:105E9700FEA3E0FFEF4E6021AE56AF5790000AE039
:105EA700FCA3E0FD12000374068E048F05FF126A3F
:105EB7009F90000AECF0A3EDF0900042E0601A908A
:105EC700000AE0FEA3E0FFAC56AD57EF2DFDEE3C18
:105ED700FC90000AECF0A3EDF0900042E0D39401AF
:105EE700401A90000AE0FEA3E0FFAC56AD57EF2D35
:105EF700FDEE3CFC90000AECF0A3EDF0D21DAE5491
:105F0700AF5590000AE0FCA3E0FDEFC39DEE9C4077
:105F1700159000D7E0B40104C2968002C2A074466F
:105F2700900041F0C21DA21DB3B35007900041E09D
:105F3700B55E0280159000D7E0B40104C2968002D6
:105F4700C2A07446900041F0C21D9000D9E0B4028F
:105F570002800302606D900073E0D39566506490F1
:105F67000073E0F4042566FE9000DCE08E00F5F097
:105F7700E884FF7E008F73EFC39410500CEF857396
:105F8700F0A4FDACF08D7380037573FF900073E090
:105F9700D39573400B900073E0C39573F57180033D
:105FA7007571009000F7E0D3957140069000F7E017
:105FB700F5719000F8E0C3957150069000F8E0F590
:105FC700718071900073E0C39566FE9000DCE08EEF
:105FD70000F5F0E884FF7E008F73EFC39410500C38
:105FE700EF8573F0A4FDACF08D7380037573FF85A7
:105FF700735B755A00900073E0255BFFAE5A500142
:106007000E8E5A8F5B74FFBE0009D39F4005855BD8
:106017007180037571FF9000F7E0D395714006908A
:1060270000F7E0F5719000F8E0C395715006900015
:10603700F8E0F571A20DB3B3500D900074E0FE9037
:1060470000E4E0D39E5002800A7407900050F0C22B
:10605700A2801375A710E5CDC395714004C2A28035
:1060670002D2A275A700E56FC39409500AA2EDB347
:106077004005C2ED123050AE54AF557410C39F7433
:10608700279E400C900072E0C3945A40030262F1CD
:10609700A212B340091242157406900050F0A220D4
:1060A700B34008E5B54404F5B58006E5B554FBF5FE
:1060B700B5A214B3500EE561D394334007E561C32D
:1060C70094CC40028041900109E0B40214120E26DC
:1060D70090007AE075F050A4FFAEF08E5C8F5D8083
:1060E7000F900085E075F050A4FFAEF08E5C8F5DD9
:1060F700E55D455C6011E5B54401F5B5742B90008D
:1061070071F012431BD214900072E0D39401400740
:10611700E561C3941A40028002C2149006C8E06089
:10612700031224EAA22D300301B35017A22DB34066
:1061370008E5B54408F5B58006E5B554F7F5B5A209
:106147002D92039006CCE060031225C6A22E3004E0
:1061570001B35017A22EB34008E5B54402F5B58048
:1061670006E5B554FDF5B5A22E92049006D0E06081
:10617700031226B6A22F300501B3500FA22FB3404A
:1061870004D2978002C297A22F92059006D4E060AE
:1061970003122792A230300601B3500FA230B3404A
:1061A70004D2A28002C2A2A23092069006D8E06072
:1061B7000312286EA231300701B3500FA231B3404A
:1061C70004D2A18002C2A1A23192079006DCE0604E
:1061D7000312294AA232300801B35017A232B34042
:1061E70008E5B54440F5B58006E5B554BFF5B5A259
:1061F7003292089006E0E06003122A26A2333009A3
:1062070001B35017A233B34008E5B54480F5B58014
:1062170006E5B5547FF5B5A23392099006E4E06030
:1062270003122B02A234300A01B3500FA234B34039
:1062370004D2928002C292A234920A9006E8E060E9
:1062470003122BDEA235300B01B3500FA235B3403A
:1062570004D2878002C287A235920B9006ECE060D9
:1062670003122CBAA236300C01B3500FA236B3403A
:1062770004D2908002C290A236920C900072E0C3C2
:10628700945A5010E56FB40909900072E004F07554
:106297006F00803BE56FB40903756F007555007596
:1062A7005400758D00758B00756400900071E0C314
:1062B70094415008900071E004F08006744190000A
:1062C70071F0900071E0B44106E5B554FEF5B59064
:1062D7000072E0D394014007E56AC394414002800D
:0D62E70009740E900050F0124215024AE2B8
:106387000000010001400160018001A001C001E09F
:1063970002000300039603B603D603F404000500C6
:1063A7000512052405360548055A056C057E059036
:1063B70005A805C005DE0600061406280646066E73
:1063C70006AE05CF00FF013F015F017F019F01BFBF
:1063D70001DF01FF02FF039503B503D503F303FFB5
:1063E70004FF05110523053505470559056B057D8F
:1063F700058F05A705BF05CE05F106130627064538
:10640700066D06AD06ED05DD0FAA0FA50F9F0F9AC6
:106417000F940F8D0F870F800F780F710F680F6024
:106427000F570F4E0F450F3B0F300F250F1A0F0E4B
:106437000F020EF50EE80EDB0ECC0EBE0EAE0E9F53
:106447000E8E0E7D0E6C0E5A0E470E340E200E0C5D
:106457000DF70DE20DCB0DB50D9D0D850D6D0D5491
:106467000D3A0D200D050CE90CCE0CB10C940C76F1
:106477000C580C3A0C1B0BFB0BDB0BBB0B9A0B7969
:106487000B570B350B130AF10ACE0AAB0A870A64BE
:106497000A400A1C09F809D409B0098C096709439D
:1064A700091F08FB08D608B2088E086A08460823A1
:1064B70007FF07DC07B9079607730751072F070D73
:1064C70006EC06CA06AA068906690649062A060AC6
:1064D70005EC05CD05B0059205750558053C052069
:1064E700050504EA04CF04B5049C04820469045139
:1064F70004390422040B03F403DE03C803B2039D2B
:10650700038903750361034D033B03280316030443
:1065170002F202E102D102C002B002A0029102829D
:106527000273026502570249023C022F0222021639
:10653700020901FD01F201E601DB01D001C601BB41
:1065470001B101A7019D0194018B018201790170BD
:1065570001680160015801500148014101390132C8
:10656700012B0125011E01180111010B010500FF77
:1065770000FA0FA60FA00F990F920F8B0F840F7CB5
:106587000F740F6B0F620F580F4E0F430F380F2CFE
:106597000F1F0F120F050EF70EE80ED80EC80EB715
:1065A7000EA50E930E800E6C0E580E420E2C0E1575
:1065B7000DFD0DE40DCB0DB10D950D790D5D0D3F65
:1065C7000D200D010CE10CC00C9E0C7C0C590C35F8
:1065D7000C100BEA0BC40B9E0B760B4F0B260AFD18
:1065E7000AD40AAA0A800A550A2A09FF09D409A85F
:1065F700097C0950092508F908CD08A10875084A3A
:10660700081E07F307C8079D07730749072006F702
:1066170006CE06A6067E06570630060A05E405BF1F
:10662700059B057705540532051004EF04CE04AE2B
:10663700048F047104530435041903FD03E203C7EF
:1066470003AD0394037B0363034B0334031E030867
:1066570002F302DE02CA02B602A30291027F026DB2
:10666700025C024C023C022C021D020E020001F2E7
:1066770001E401D701CA01BE01B101A6019A018F48
:106687000185017A01700166015D0153014A0141EB
:10669700013901310129012101190112010B0104FD
:1066A70000FD00F700F000EA00E400DE00D900D3A7
:1066B70000CE00C900C400BF00BA00B500B100ADEC
:1066C70000A800A400A0009C009900950091008EEE
:0C66D700008A008700840081007E007BA8
:10009E007547009007C5E4F0A3F075310075300088
:1000AE00754D00754E00C238D23974FE9007C7F8F0
:1000BE00E4F0E8A3F074FE9007C9F8E4F0E8A3F0CA
:1000CE0074FE9007D3F0745A9007D4F0745A9007C8
:1000DE00D5F0D23AC22CC23CC23722750B00750A3B
:1000EE0000AE0AAF0BAC08AD09EDC39FEC9E4016F7
:1000FE0074FF126A8F75CF01780B740126F65004C7
:10010E0018E436F650DB2290004CE0B4AA1C90079F
:10011E0081E0B43C159007C1E0FEA3E0FFEF4E6016
:10012E0009741EBE0004D39F5003020243755D0086
:10013E00755C0075F8099007C1E0FEA3E0FF740737
:10014E006F4E6006740E6F4E7006743A900781F013
:10015E009007C1E0FEA3E0FF7408BE001ED39F40CF
:10016E001A7E017F089007C1E0FCA3E0FD1DBDFFD4
:10017E00011C1200038E5A8F5B801F9007C1E0FE98
:10018E00A3E0FF7408126AF38F048E057E017F08C8
:10019E00CDCCCD1200038E5A8F5BAE5CAF5D740C6E
:1001AE00D39F74019E500302023EA2F9B3407EE536
:1001BE005D455C700375A382AE5CAF5D74016F4EDE
:1001CE00700375A300AE5CAF5D74026F4E700D9040
:1001DE0007C2E075F002A4FDACF08DA3AE5CAF5D7E
:1001EE0074036F4E700375A300AE5CAF5D7403BEF7
:1001FE0000039F5013AC5AAD5BED2FFFEC3EFE900B
:10020E00007D126AD6E0F5A3AE5CAF5DEFB40B09CC
:10021E00EEB401057414126A8FAE5CAF5DEFB40BD1
:10022E0007EEB4010375F80D785C126B030201A89A
:10023E0090004CE4F022755D00755C0075F8099035
:10024E0007C1E0FEA3E0FF7408BE001ED39F401A54
:10025E007E017F089007C1E0FCA3E0FD1DBDFF01FC
:10026E001C1200038E5A8F5B801F9007C1E0FEA305
:10027E00E0FF7408126AF38F048E057E017F08CDAD
:10028E00CCCD1200038E5A8F5BAE5CAF5D7411D372
:10029E009F74019E5003020374A2F9B3500302032C
:1002AE0071E55D455C700375A3D2AE5CAF5D740104
:1002BE006F4E700375A300AE5CAF5D74026F4E702F
:1002CE000D9007C2E075F002A4FDACF08DA3AE5CFC
:1002DE00AF5D74036F4E700375A300AE5CAF5D74BB
:1002EE00046F4E700375A300AE5CAF5D74056F4E68
:1002FE00700375A300AE5CAF5D74066F4E70037530
:10030E00A300AE5CAF5D74076F4E700375A300AEB5
:10031E005CAF5D74086F4E700375A300AE5CAF5D8D
:10032E007408BE00039F5016AC5AAD5BED2FFFEC68
:10033E003EFE900078126AD6E5A3F075A300AE5C7F
:10034E00AF5DEFB41009EEB401057414126A8FAEEE
:10035E005CAF5DEFB41007EEB4010375F80D785C79
:10036E00126B0302029722755D00755C0075F80929
:10037E00AE5CAF5D7417BE0004D39F500302044DF4
:10038E00A2F9B3500302044AE55D455C700375A300
:10039E00D2AE5CAF5D74016F4E700375A300AE5CA0
:1003AE00AF5D74026F4E700D9007C2E075F002A43F
:1003BE00FDACF08DA3AE5CAF5D74036F4E70037534
:1003CE00A300AE5CAF5D74046F4E700375A300AEF8
:1003DE005CAF5D74056F4E700375A300AE5CAF5DD0
:1003EE0074066F4E700375A300AE5CAF5D74076F3D
:1003FE004E700375A300AE5CAF5D74086F4E700354
:10040E0075A300AE5CAF5D7408BE00039F500C90E8
:10041E00005A126AD6E5A3F075A300AE5CAF5D7408
:10042E00166F4E70057414126A8FAE5CAF5D741643
:10043E006F4E700375F80D785C126B0302037E220B
:10044E0090004CE0B4AB0280030204E8755D0075C9
:10045E005C0075F809AE5CAF5D7412BE007CD39F74
:10046E004078A2F9B34070E55D455C700375A382D8
:10047E00AE5CAF5D74016F4E700375A300AE5CAFE2
:10048E005D74026F4E700D9007C2E075F002A4FD10
:10049E00ACF08DA3AE5CAF5D74036F4E700375A3AD
:1004AE0000AE5CAF5D7403BE00039F500990005F09
:1004BE00126AD6E0F5A3AE5CAF5D74116F4E700597
:1004CE007414126A8FAE5CAF5D74116F4E7003754B
:1004DE00F80D785C126B03020463229007D0E4F0EF
:1004EE0074649007C1F8E4F0E8A3F012037574C8C1
:1004FE009007C1F8E4F0E8A3F074FF90005AF0748E
:10050E00FF90005BF074FF90005CF074009000545C
:10051E00F074FF90005DF0740090005FF074019035
:10052E000060F0900066E0B4371A900063E090002F
:10053E005AF0900064E090005BF0900065E090004F
:10054E005CF080469007D07401F074659007C1F896
:10055E00E4F0E8A3F012037574C89007C1F8E4F054
:10056E00E8A3F0900066E0B4371A900063E09000C4
:10057E005AF0900064E090005BF0900065E090000F
:10058E005CF0800674029007D0F09007D1E4F0740E
:10059E00669007C1F8E4F0E8A3F012037574C890F2
:1005AE0007C1F8E4F0E8A3F0900065E0B4371290CC
:1005BE000063E0900054F0900064E090005DF080E5
:1005CE00769007D17401F074679007C1F8E4F0E8F3
:1005DE00A3F012037574C89007C1F8E4F0E8A3F015
:1005EE00900065E0B43712900063E0900054F090F4
:1005FE000064E090005DF0803E74029007D1F074CC
:10060E00689007C1F8E4F0E8A3F012037574C8907F
:10061E0007C1F8E4F0E8A3F0900065E0B43712905B
:10062E000063E0900054F0900064E090005DF08074
:10063E000674039007D1F022E54E64046006E59936
:10064E0064FF60028031A2384004D2388027E54E24
:10065E00600874E6254E900050F0E54D600874F089
:10066E00254D900050F0E54EB4010280FE754E000F
:10067E00754D00C2388002C238E54E90384AF828CF
:10068E002873754E00E599B4FF03754D01E599B4D5
:10069E00FE03754D02E599B4FD03754D03E599B45E
:1006AE00FC03754D04E599B4FA03754D05E599B44F
:1006BE00FB06754E01124215E599B4F906754E0406
:1006CE00124215E599D394E54007E599C394F0409D
:1006DE0002801685994F754E027E017F00E54FC34D
:1006EE0094E6126AAF8E328F339007C5E4F0A3F012
:1006FE00E599D394C44007E599C394E64002802857
:10070E0085994F754E0374E5C3954FF533753200D9
:10071E00AE32AF33906387126A7EE493F87401931E
:10072E009007C5C8F0A3C8F0D299020C569000638A
:10073E00E07005A22AB3400280429007C5E0FEA3F6
:10074E00E0FF74FFBE00039F5009EFC39446EE9482
:10075E000640119007C5E0FEA3E0FFEFD3946DEEC7
:10076E00940640139007C5E0FEA3E0FF90008112AF
:10077E006AD6E599F0800385997480119007C5E0DB
:10078E00FEA3E0FF900081126AD6E599F09007C5AE
:10079E00126ABD9007C5E0FEA3E0FFEFB40106EEBE
:1007AE00B4070280030209FD900781E0B43C028089
:1007BE00030209FDA22A50030208E8C29C900063BE
:1007CE00E090011FF0900064E090008EF0900065C4
:1007DE00E09000AEF0900066E09000D7F0900067D9
:1007EE00E0900083F0900068E09000C9F0900069FE
:1007FE00E09000E7F090006AE09000BBF090006B94
:10080E00E09000D9F090006CE0900109F090006D3E
:10081E00E090016DF090006EE090016EF090006F30
:10082E00E090016FF0123BC1900075E09000F0F087
:10083E00900076E09000A7F0900077E09000A8F08E
:10084E0074639007C1F8E4F0E8A3F074AB90004C29
:10085E00F012044E90004CE4F07464F50975080033
:10086E001200E9A21F4039757301E573D394075046
:10087E002DE5739007C1F8E4F0E8A3F074AA900098
:10088E004CF0120115E573C39407500A7464F50910
:10089E007508001200E97873740126F650CC803783
:1008AE00757308E573D3940E502DE5739007C1F858
:1008BE00E4F0E8A3F074AA90004CF0120115E57371
:1008CE00C3940E500A7464F5097508001200E97895
:1008DE0073740126F650CC0209E7C29C90011FE00A
:1008EE00900063F090008EE0900064F09000AEE017
:1008FE00900065F09000D7E0900066F0900083E0E5
:10090E00900067F09000C9E0900068F09000E7E07A
:10091E00900069F09000BBE090006AF09000D9E082
:10092E0090006BF0900109E090006CF07400900064
:10093E006DF0740090006EF0740090006FF07463B0
:10094E009007C1F8E4F0E8A3F074AB90004CF012FD
:10095E00044E90004CE4F07464F509750800120022
:10096E00E9757301E573D394075026E5739007C1BB
:10097E00F8E4F0E8A3F074AA90004CF0120115749C
:10098E0064F5097508001200E97873740126F650B3
:10099E00D3D29C7599FB743C900781F0757308E572
:1009AE0073D3940E5026E5739007C1F8E4F0E8A3D4
:1009BE00F074AA90004CF01201157464F5097508D4
:1009CE00001200E97873740126F650D374C89007AC
:1009DE00C1F8E4F0E8A3F080FE74C89007C1F8E413
:1009EE00F0E8A3F0D29C754E00754D007599FB0290
:1009FE000C569007C5E0FEA3E0FFEF4E70068599FA
:100A0E00317530009007C5E0FEA3E0FF74016F4E14
:100A1E00701BAC30AD31AA32AB33ED2BFBEC3AFA96
:100A2E008A068B07900081126AD6E599F09007C569
:100A3E00126ABD9007C5E0FEA3E0FF74026F4E7010
:100A4E0021AC30AD3174566D4C7006E54F64E660E6
:100A5E00028003124215123BC1854F99754E0075E7
:100A6E004D00020C569007C5E0FEA3E0FF900081FA
:100A7E00126AD6E599F09007C5126ABD9007C5E0D7
:100A8E00FEA3E0FFAC32AD338F028E038C068D07D2
:100A9E009063CB126A7EE493F9740193FEEAD39EBF
:100AAE00EB994009854F99754E00754D00020C5615
:100ABE009007C5E0FEA3E0FF900081126AD6E5998B
:100ACE00F09007C5126ABD9007C5E0FEA3E0FFEFE8
:100ADE00B40006EEB401028003020C5690005CE0F6
:100AEE00D394C7400B90005CE0C394C8F550801AB5
:100AFE0090005CE0D39463400B90005CE0C3946480
:100B0E00F550800690005CE0F550E55075F002A4BB
:100B1E00FFAEF08F73EF900081126AE1EFFCE0FD03
:100B2E00EC900084126AE1EDFCE0FDEC2DB5500274
:100B3E008003020C470FEF900081126AE1E573FF0C
:100B4E00E0FCEF900085126AE1ECFFE0FCEFC39C45
:100B5E00B550028003020C47E573900083126AE1E0
:100B6E00E573FFE0FCEF900086126AE1ECFFE0FC1B
:100B7E00EF2CB550028003020C47E57390008712EC
:100B8E006AE1E0C39550900063F0E573900088121F
:100B9E006AE1E0C39550900064F0E573900089120D
:100BAE006AE1E0C39550900065F07400900066F025
:100BBE0074FF900067F0E57390008B126AE1E0C35A
:100BCE009550900068F0E57390008C126AE1E0C3D6
:100BDE009550900069F0E57390008D126AE1E0C3C4
:100BEE00955090006AF0E57390008A126AE1E0C3B6
:100BFE0095509007C1F8E4F0E8A3F074AB90004C68
:100C0E00F012044E7464F5097508001200E990079D
:100C1E00C1126ABD12044E7464F509750800120003
:100C2E00E99007C1126ABD12044E7599F97464F504
:100C3E00097508001200E980FE7599FF7464F509C4
:080C4E007508001200E980FEA8
:0F384A0002069002073B020A00020A73020ABE3E
:100C560022E54D903859F8282873020D699007C58A
:100C6600E0FEA3E0FF900052126AD6E0F5999007E5
:100C7600C5126ABD9007C5E0FEA3E0FF74116F4E72
:100C86007003754D00020D69856E99020D69900716
:100C9600C5E0FEA3E0FF900081126AD6E0F599EF69
:100CA600B40107EEB40703754D009007C5126ABD7F
:070CB600020D699007C6E082
:0F385900020C60020C63020C8E020C94020CB97C
:100CBD00903A0CF8282873855399020D5E855F993B
:100CCD00020D5E856199020D5E856599020D5E8549
:100CDD006799807D85689980788569998073856A23
:100CED0099806E90001AE0F5998066A239B340079D
:100CFD007599FAC2398041A229B3400575990F80C3
:100D0D00359007D0E0600A9007D0E024DCF599809B
:100D1D00169007D1E0600A9007D1E024DEF59980A6
:100D2D0006900050E0F599900050E4F09007D0E463
:100D3D00F09007D1E4F0C2298017856B9980128558
:100D4D006699800D856C9980087599FC8003754DA9
:010D5D000095
:103A0C00020CC4020CCA020CD0020CD6020CDC0252
:103A1C000CE1020CE6020CEB020CF0020CF8020DAD
:0D3A2C0047020D4C020D51020D56020D5BBC
:0B0D5E009007C5126ABD8003123A39ED
:03386800020D66E8
:100D690022E537255BFFAE5A50010E900081126AC9
:100D7900D6E0F538E537255BFFAE5A50010E0FBFB7
:100D890000010E900081126AD6E0F539853F3BE5F6
:100D990038B539058538378041E539D39538401D4F
:100DA900E539C39538853AF0A4FFAEF0E53B8E04EA
:100DB9008F05FF126A9FED2538F537801DE538C389
:100DC9009539853AF0A4FFAEF0E53B8E048F05FF17
:100DD900126A9FEDF4042538F53722E539D39538A1
:100DE900401DE539C39538853AF0A4FFAEF0E53BDF
:100DF9008E048F05FF126A9FED2538F537801DE5B2
:100E090038C39539853AF0A4FFAEF0E53B8E048FDF
:100E190005FF126A9FEDF4042538F5372290008703
:100E2900E0B40170E56775F00A84FF7E008F37E54D
:100E39006775F00A84ADF07C008D3A753F0A755AE2
:100E490005755B24E537C394115005120D6A8006B8
:100E59009005B6E0F537E53790007AF0E56775F06B
:100E69000A84FF7E008F37E56775F00A84ADF07C50
:100E7900008D3A753F0A755A05755B5AE537C39473
:100E8900115005120D6A80069005ECE0F537E5373B
:100E9900900012F022900087E0B4016AE56775F0CE
:100EA9000A84FF7E008F37E56775F00A84ADF07C10
:100EB900008D3A753F0A755A05755B36E537C39457
:100EC900115005120D6A80069005C8E0F53785377F
:100ED9004BE56775F00A84FF7E008F37E56775F08B
:100EE9000A84ADF07C008D3A753F0A755A05755B29
:100EF90048E537C394115005120D6A80069005DA4A
:100F0900E0F53785374C22E55F75F00484FF7E00F4
:100F19008F37E55F75F00484ADF07C008D3A753F3D
:100F290004755A01755B00E537C3943F5005120DEE
:100F39006A80069001C0E0F5378537297528009049
:100F4900004FE075F020A4FFAEF09000D2E08E04CF
:100F59008F05FF126A9F8D379000BAE0D3955F50D5
:100F6900030210169000DEE0D3955F4010ED90016A
:100F7900C1126AE1E0F52B752A000210139000A94D
:100F8900E0D3955F4043E5379001C1126AE1E0F58E
:100F990038E5379001E1126AE1E0F5399000DEE0C9
:100FA900F404255FF53A9000A9E0FE9000DEE0F434
:100FB900042EF53BE538B539058538378003120D20
:100FC900E485372B752A008041E5379001E1126AE3
:100FD900E1E0F538E537900201126AE1E0F5399070
:100FE90000A9E0F404255FF53A9000BAE0FE90000C
:100FF900A9E0F4042EF53BE538B539058538378085
:1010090003120DE485372B752A000210BD9000E10B
:10101900E0D3955F5011E537900241126AE1E0F59E
:101029002B752A000210BD9000AAE0D3955F5043AA
:10103900E537900221126AE1E0F538E5379002417F
:10104900126AE1E0F5399000AAE0F404255FF53A67
:101059009000E1E0FE9000AAE0F4042EF53BE538AB
:10106900B539058538378003120DE485372B752A84
:10107900008041E537900201126AE1E0F538E53771
:10108900900221126AE1E0F5399000BAE0F40425F2
:101099005FF53A9000AAE0FE9000BAE0F4042EF55C
:1010A9003BE538B539058538378003120DE48537B6
:1010B9002B752A00229000F2E0F53C753F11755A14
:1010C90002755B00AE52AF53E53C75F00FA4FDAC61
:1010D900F0EDD39FEC9E4021E53C8E048F05FF1275
:1010E9006A9FED75F010A4FFAEF0E55F75F011840D
:1010F900FD7C00ED2FF53D800EE55F75F01184FF55
:101109007E00EF24F0F53D853D37E55F75F01184EC
:10111900AFF07E008F3A120D6A85373EAE52AF535B
:101129009000F2E075F00FA4FDACF0EDD39FEC9EBA
:101139004028755A02755B10853D37120D6A853E48
:1011490038853739AE52AF53E53C8E048F05FF120F
:101159006ACA8D3A853C3B120DE48537297528000A
:10116900752B64752A00229000F2E0F53C753F1159
:10117900755A02755B00AE52AF53E53C75F00FA48A
:10118900FDACF0EDD39FEC9E4021E53C8E048F052C
:10119900FF126A9FED75F010A4FFAEF0E56175F0DE
:1011A9001184FD7C00ED2FF53D800EE56175F01190
:1011B90084FF7E00EF24F0F53D853D37E56175F04C
:1011C9001184AFF07E008F3A120D6A85373EAE5218
:1011D900AF539000F2E075F00FA4FDACF0EDD39F92
:1011E900EC9E4028755A02755B10853D37120D6AD1
:1011F900853E38853739AE52AF53E53C8E048F05AD
:10120900FF126ACA8D3A853C3B120DE48537297570
:101219002800E56B6017E56BC394FE50109000E65B
:10122900E0B402099000D4E0D3940B50028017AEC9
:1012390028AF29E56B126AAF74E78E048F05FF1298
:101249006A9F8C288D299000BCE0B40453E55F7532
:10125900F00484FF7E008F37E55F75F00484ADF0FC
:101269007C008D3A753F04755A01755B00E537C3FB
:10127900943F5005120D6A80069001C0E0F537AE23
:1012890028AF29E537126AAF74648E048F05FF12FF
:101299006A9FAE28AF29EF2DFDEE3CFC8C288D29E5
:1012A900752B64752A0022900087E0B40146E56732
:1012B90075F00A84FF7E008F37E56775F00A84AD03
:1012C900F07C008D3A753F0A755A05755B00E53764
:1012D900C394115005120D6A8006900592E0F53706
:1012E900AE2AAF2BE5372FFF50010E7464126AF353
:1012F9008E2A8F2B900088E0B40146E56875F00AC4
:1013090084FF7E008F37E56875F00A84ADF07C00B4
:101319008D3A753F0A755A05755B6CE537C39411AB
:101329005005120D6A80069005FEE0F537AE2AAF2A
:101339002BE5372FFF50010E7464126AF38E2A8F42
:101349002B900097E0B40249E56AC3944175F00512
:1013590084FF7E008F37E56A75F00584ADF07C0067
:101369008D3A753F05755A06755B00E537C39413C9
:101379005005120D6A8006900694E0F537AE2AAF43
:101389002BE5372FFF50010E7464126AF38E2A8FF2
:101399002B9000D9E0B40202800302144FE55F7577
:1013A900F01584FF7E008F37E55F75F01584ADF089
:1013B9007C008D3A753F15755A03755BF4E537C3A3
:1013C900940B5005120D6A8006900480E0F537E50C
:1013D9003775F0FFA4FFAEF09000DAE08E048F05B8
:1013E900FF126A9FED900073F0E56675F078A4FF2F
:1013F900AEF074FF8E048F05FF126A9F8C5A8D5BC5
:1014090074028C068D071200398F37AC5AAD5B74A4
:1014190004FF126ACA8D3A753F04755A06755B282E
:10142900E537C3941D5005120D6A80069006C6E083
:10143900F537AE2AAF2BE5372FFF50010E74641232
:101449006AF38E2A8F2B900086E0B4025DE5617500
:10145900F064A4FFAEF074081200398E5C8F5D74DD
:10146900058E048F05FF126A9F8D37AE5CAF5D74E0
:10147900058E048F05FF126ACA8D3A753F05755AA4
:1014890005755BDEE537C394135005120D6A8006B6
:10149900900672E0F537AE2AAF2BE5372FFF5001E2
:1014A9000E7464126AF38E2A8F2B9000C8E0703C88
:1014B90090004FE075F00584FF7E008F3790004F54
:1014C900E075F00584ADF07C008D3A753F05755ADD
:1014D90005755BC0E537C3941D5005120D6A80067A
:1014E90090065EE0F537E53790007BF02290008F9B
:1014F900E0B401179007CCE0252BFFAE2A50010E6E
:101509009000E3E0126AF38E2A8F2B900107E0B472
:101519000114900108E0A852B8000495535007E55A
:101529005FC39560400280129000B1E0252BFFAEA9
:101539002A50010E8E2A8F2B802F90008FE0B40342
:1015490016A22CB3B350109007CFE0C39405A8524C
:10155900B800069553400280109000B1E0252BFF9A
:10156900AE2A50010E8E2A8F2B900089E0B4020218
:1015790080030218F490008CE0602FE567D394464D
:101589004028900013E0FEA3E0FF9000C7E075F04B
:1015990003A4FDACF0EFD39DEE9C400E9000EBE070
:1015A900A852B80005D3955350030218F49000BC13
:1015B900E0B40302800302175885615B755A0090F5
:1015C9000093E0A852B800049553500E900094E09F
:1015D900A85AB80005D3955B5003021755E5617504
:1015E900F002A4FFAEF074158E048F05FF126A9FF6
:1015F9008C068D07900611126AD6FEE0FFEE900068
:101609008BE0FEEF8E0088F0A4FFAEF074648E04C8
:101619008F05FF126A9F8C5A8D5B90004FE075F021
:1016290018A4FFAEF09000D2E08E048F05FF126A75
:101639009F8C068D07900629126AD6AE5AAF5BE0D9
:10164900126AAF74648E048F05FF126A9F8C5A8DDB
:101659005BE565A85AB80077D3955B4072E565C329
:10166900955BFFE4955AFE8E5A8F5B7428BE000382
:101679009F500C755B28755A00740D900050F0AEA0
:101689005AAF5B90008CE0126AAF74288E048F0504
:10169900FF126A9F8C5A8D5BAE28AF29740A8E049B
:1016A9008F05FF126A9F8D068C07AC5AAD5BCFCEB2
:1016B900CF120003740A8E048F05FF126A9F8C5A99
:1016C9008D5BAE28AF29126AFB8E288F29807DE5B4
:1016D90065A85AB80004955B5072AE5AAF5BE565D0
:1016E900126AF38E5A8F5B7428BE00039F500C75E3
:1016F9005B28755A00740D900050F0AE5AAF5B909C
:10170900008CE0126AAF74288E048F05FF126A9F5D
:101719008C5A8D5BAE28AF29740A8E048F05FF128F
:101729006A9F8D068C07AC5AAD5BCFCECF120003F2
:10173900740A8E048F05FF126A9F8C5A8D5BAE283E
:10174900AF29EF2DFDEE3CFC8C288D290218F49071
:1017590000D4E0855FF0A4FFAEF07405126AAF749F
:10176900071200398E5A8F5B900093E0A852B80097
:101779000495535012900094E075F002A4FDACF06A
:10178900EFC39DEE9C40030218F4E55F75F00B84EE
:10179900FF7E00900611126AD6FEE0FFEE90008BE4
:1017A900E0FEEF8E0088F0A4FFAEF074648E048F23
:1017B90005FF126A9F8C5A8D5B90004FE075F018F7
:1017C900A4FFAEF09000D2E08E048F05FF126A9F4D
:1017D9008C068D07900629126AD6AE5AAF5BE012C5
:1017E9006AAF74648E048F05FF126A9F8C5A8D5BF1
:1017F900E565A85AB80077D3955B4072E565C3954E
:101809005BFFE4955AFE8E5A8F5B7428BE00039FD6
:10181900500C755B28755A00740D900050F0AE5A43
:10182900AF5B90008CE0126AAF74288E048F05FFBD
:10183900126A9F8C5A8D5BAE28AF29740A8E048F69
:1018490005FF126A9F8D068C07AC5AAD5BCFCECFD0
:10185900120003740A8E048F05FF126A9F8C5A8D39
:101869005BAE28AF29126AFB8E288F29807DE5653A
:10187900A85AB80004955B5072AE5AAF5BE5651281
:101889006AF38E5A8F5B7428BE00039F500C755BF8
:1018990028755A00740D900050F0AE5AAF5B900055
:1018A9008CE0126AAF74288E048F05FF126A9F8C30
:1018B9005A8D5BAE28AF29740A8E048F05FF126A10
:1018C9009F8D068C07AC5AAD5BCFCECF1200037447
:1018D9000A8E048F05FF126A9F8C5A8D5BAE28AF62
:1018E90029EF2DFDEE3CFC8C288D29229000E7E0A4
:1018F900B4026AE55F75F00884FF7E008F37E55F03
:1019090075F00884ADF07C008D3A753F08755A0171
:10191900755BE0E537C3943F5005120D6A80069068
:101929000280E0F53785372D752C00AE2CAF2DAC34
:101939002AAD2B12000374648E048F05FF126A9F6F
:101949008C2C8D2D900084E08C068D07126AAF7463
:10195900648E048F05FF126A9F8C2C8D2DAE28AFE3
:1019690029AC2AAD2B12000374648E048F05FF1273
:101979006A9F8C288D29900084E08C068D07126A55
:10198900AF74648E048F05FF126A9F8C288D29A27B
:101999000D401DAE52AF537405BE00039F5002D2D5
:1019A9000DE561D394CC4008D2017411900050F038
:1019B9009000E6E0B402089000D4E0640B60028075
:1019C90035AE28AF29E56B126AAF74E78E048F052F
:1019D900FF126A9F8C288D299000E7E0B40217AEA8
:1019E9002CAF2DE56B126AAF74E78E048F05FF12D9
:1019F9006A9F8C2C8D2D9000A6E05402601B9000EC
:101A09009DE0A852B80012D39553400DA20DB3B36F
:101A19005007E561C3949A40028028AE34AF3590EF
:101A2900009BE075F002A4FDACF0EF2DFDEE3CFC4F
:101A390074022DFD50010CE561BC0007D39D4003E4
:101A4900754301856135753400E5437003021B3820
:101A59009000F9E0C395435003021B2A900109E065
:101A6900C394025076E56775F00A84FF7E009005FD
:101A790081126AD6E0F55B755A00AE5AAF5B9000E9
:101A89009CE0126AAF74648E048F05FF126A9F8C02
:101A99005C8D5D9000F9E004C395438C068D0712B7
:101AA9006AAF9000F9E08E048F05FF126A9F8C5C83
:101AB9008D5DAE28AF29EF2DFDEE3CFC8C288D29DC
:101AC9009000E7E0B40212AE2CAF2DAA5CAB5DEF3B
:101AD9002BFBEE3AFA8A2C8B2D80469000F9E00414
:101AE900C39543854BF0A4FFAEF09000F9E08E0456
:101AF9008F05FF126A9F8C5C8D5DAE28AF29EF2D93
:101B0900FDEE3CFC8C288D299000E7E0B40212AE72
:101B19002CAF2DAA5CAB5DEF2BFBEE3AFA8A2C8B2E
:101B29002D05439000F9E0C3954350037543009098
:101B390000A6E05401601B90009AE0A852B8001278
:101B4900D39553400DA20DB3B35007E55FC394CCB1
:101B590040028025900098E075F003A4FFAEF0E5FF
:101B6900402FFF50010E74032FFF50010EE55FBE99
:101B79000007D39F4003754401855F40E544700326
:101B8900021C6B9000FAE0C395445003021C5D905F
:101B99000109E0C394025076E56775F00A84FF7E77
:101BA90000900581126AD6E0F55B755A00AE5AAF0E
:101BB9005B900099E0126AAF74648E048F05FF127E
:101BC9006A9F8C5C8D5D9000FAE004C395448C0695
:101BD9008D07126AAF9000FAE08E048F05FF126A32
:101BE9009F8C5C8D5DAE28AF29EF2DFDEE3CFC8C02
:101BF900288D299000E7E0B40212AE2CAF2DAA5C23
:101C0900AB5DEF2BFBEE3AFA8A2C8B2D80469000C8
:101C1900FAE004C39544854CF0A4FFAEF09000FAB5
:101C2900E08E048F05FF126A9F8C5C8D5DAE28AF34
:101C390029EF2DFDEE3CFC8C288D299000E7E0B4BE
:101C49000212AE2CAF2DAA5CAB5DEF2BFBEE3AFA7C
:101C59008A2C8B2D05449000FAE0C39544500375F6
:101C690044009000FCE02529FFAE2850010E8E2883
:101C79008F299000ABE0A828B80004952950099055
:101C890000ABE0F5297528009000E7E0B4020D905B
:101C990000ABE0A82CB80006952D40028009900001
:101CA900ABE0F52D752C00229000E7E0B40102802D
:101CB90003021DBCA20DB35003021DBA9000B2E08D
:101CC900B40168AE28AF29AC52AD53120003743C7D
:101CD9008E048F05FF126A9F9000C2E0BC00109D20
:101CE900400D9000C4E0A828B8000495295002D2FC
:101CF90002AE28AF29AC52AD53120003743C8E04D6
:101D09008F05FF126A9F9000C2E0C3940ABC0015B8
:101D1900D39D40119000C4E0C39405A828B80005DC
:101D2900D3952950028002C2028068AE28AF29AC3F
:101D390052AD5312000374788E048F05FF126A9F07
:101D49009000C2E0BC00109D400D9000C4E0A8289E
:101D5900B8000495295004D2028038AE28AF29ACC6
:101D690052AD5312000374788E048F05FF126A9FD7
:101D79009000C2E0C3940ABC0015D39D40119000A5
:101D8900C4E0C39405A828B80005D395295002805A
:101D990002C202A202B34019AE28AF299000C3E0E3
:101DA900126AAF74648E048F05FF126A9F8C288DA6
:101DB900298002C202A200B34006A201B3B35009AE
:101DC900900019E4F0A3F08024AE28AF297400D361
:101DD9009F74019E400C900019E528F0A3E529F0B5
:101DE900800B74FF900019F8E4F0E8A3F09000C9A3
:101DF900E0D39402400C9000B4E07006A20DB3B396
:101E09004002801AAE28AF297402126AAF8E288F59
:101E190029AE2CAF2D7402126AAF8E2C8F2D900033
:101E2900B2E0B4011AAE28AF297402126AAF8E2843
:101E39008F29AE2CAF2D7402126AAF8E2C8F2DAE66
:101E490028AF29745E126AAF740A8E048F05FF12D7
:101E59006A9F8C288D299000E7E0B40217AE2CAF59
:101E69002D745E126AAF740A8E048F05FF126A9F81
:101E79008C2C8D2DAE28AF297402BE000AD39F4049
:101E890006752902752800AE2CAF2D7402BE000A12
:101E9900D39F4006752D02752C00900017E528F098
:101EA900A3E529F02290004FE0900381126AE1E056
:101EB900F54175426490004FE0FE9000BDE0D39E6D
:101EC9004037E55F75F00884FF7E008F37E55F7561
:101ED900F00884ADF07C008D3A753F08755A03759A
:101EE9005B96E537C3941F5005120D6A800690046E
:101EF90036E0F5378537428035E55F75F00884FFB0
:101F09007E008F37E55F75F00884ADF07C008D3A6F
:101F1900753F08755A03755BB6E537C3941F5005BD
:101F2900120D6A8006900456E0F5378537422290F3
:101F390000F3E0F53C753F11755A04755B00AE522C
:101F4900AF53E53C75F00FA4FDACF0EDD39FEC9ECB
:101F59004021E53C8E048F05FF126A9FED75F01054
:101F6900A4FFAEF0E55F75F01184FD7C00ED2FF55F
:101F79003D800EE55F75F01184FF7E00EF24F0F5DA
:101F89003D853D37E55F75F01184AFF07E008F3AEE
:101F9900120D6A85373EAE52AF539000F3E075F0EB
:101FA9000FA4FDACF0EDD39FEC9E4028755A047543
:101FB9005B10853D37120D6A853E38853739AE523B
:101FC900AF53E53C8E048F05FF126ACA8D3A853CF2
:101FD9003B120DE4853741754264229000F3E0F528
:101FE9003C753F11755A04755B00AE52AF53E53C21
:101FF90075F00FA4FDACF0EDD39FEC9E4021E53CBC
:102009008E048F05FF126A9FED75F010A4FFAEF0E4
:10201900E56175F01184FD7C00ED2FF53D800EE53D
:102029006175F01184FF7E00EF24F0F53D853D37A1
:10203900E56175F01184AFF07E008F3A120D6A8563
:10204900373EAE52AF539000F3E075F00FA4FDACEC
:10205900F0EDD39FEC9E4028755A04755B10853DC1
:1020690037120D6A853E38853739AE52AF53E53C94
:102079008E048F05FF126ACA8D3A853C3B120DE426
:102089008537417542649000BCE0B4047990004FF3
:10209900E0FE9000BDE0D39E4037E55F75F008840F
:1020A900FF7E008F37E55F75F00884ADF07C008D09
:1020B9003A753F08755A03755B96E537C3941F5007
:1020C90005120D6A8006900436E0F537853742809F
:1020D90035E55F75F00884FF7E008F37E55F75F0A1
:1020E9000884ADF07C008D3A753F08755A03755B1D
:1020F900B6E537C3941F5005120D6A800690045641
:10210900E0F53785374222900087E0B4013BE56767
:1021190075F00A84FF7E008F37E56775F00A84AD94
:10212900F07C008D3A753F0A755A05755B12E537E3
:10213900C394115005120D6A80069005A4E0F53785
:10214900E5422537C39464F542900088E0B4013B29
:10215900E56875F00A84FF7E008F37E56875F00A37
:1021690084ADF07C008D3A753F0A755A05755B7E22
:10217900E537C394115005120D6A8006900610E0E8
:10218900F537E5422537C39464F542E5412542F523
:102199003690008FE0B402109007CBE02536FE9010
:1021A90000E3E0F4042EF5369000E6E0D394014014
:1021B90040E56BC394E7501D74E7C3956BFE900728
:1021C900CDE08E00F5F0E884FF7E008F37E53625F7
:1021D90037F536801CE56BC394E7FE9007CDE08E9A
:1021E90000F5F0E884FF7E008F37E536C39537F5B3
:1021F90036A20D4006E5412464F536E536D39464EC
:102209004009E536C39464F53680037536009000BD
:10221900BFE0C3953650069000BFE0F53622D200E4
:10222900900079E0A852B800049553504190007984
:10223900E0A852B800049553500375360F90007901
:10224900E004A852B800049553500375360A90006B
:1022590079E02402A852B800049553500575360553
:10226900C200900079E060067409900050F0C23C09
:102279007E017F009000C5E0126AAF9000D4E08E25
:10228900048F05FF126A9FE55FBC0017D39D4013B9
:102299009000CEE0B40204D23C8002C200740A90DD
:1022A9000050F09000C6E0C3956750159000D8E043
:1022B900A852B8000495535002C200740B90005004
:1022C900F0E567C39464501D90011EE0600D900114
:1022D9001EE0A852B80006955340028008C2007457
:1022E9000B900050F0A2004003753605900107E0FD
:1022F900B40114900108E0A852B80004955350079E
:10230900E55FC39560400280089000B0E0F5368033
:102319003A90008FE0B40306A22CB3B34002802B9D
:102329009007CFE0C39405A852B800049553500C08
:102339009000B0E0F536740C900050F09007CFE0B3
:10234900A852B8000495535002C20085366C90001B
:1023590081E02536FE90004FE075F01E84FC7F0079
:10236900EE2CF5362290004FE075F00584FF7E00D3
:102379008F3790004FE075F00584ADF07C008D3A01
:10238900753F05755A03755BD69000D2E01475F058
:102399000584FF7E00E537BE00039F5005120D6AD4
:1023A900800BE537900457126AE1E0F537E537907D
:1023B90007CEF09007CEE0FE9000C1E0C39E500822
:1023C9009000C1E09007CEF022E56775F00A84FF1E
:1023D9007E00900581126AD6E0F546E546D39464FD
:1023E9004010E546C3946475F00F84FF7E008F4664
:1023F90080037546009000A4E02546F5462290002A
:10240900BCE0C3940350269007BBE0FEA3E0FF7431
:1024190004120039E55F126AAF740F8E048F05FF4D
:10242900126A9F9007B9ECF0A3EDF080249007BBE6
:10243900E0FEA3E0FF7404120039E561126AAF748B
:102449000F8E048F05FF126A9F9007B9ECF0A3ED78
:10245900F0900097E0B40262E56AC3944175F00513
:1024690084FF7E008F37E56A75F00584ADF07C0046
:102479008D3A753F05755A06755B14E537C3941790
:102489005005120D6A80069006A8E0F5379007B945
:10249900E0FEA3E0FF740A8E048F05FF126A9FE530
:1024A900378C068D07126AAF740A8E048F05FF12E6
:1024B9006A9F9007B9ECF0A3EDF09007B9E0FEA38D
:1024C900E0FF9007BFE0FCA3E0FDEDD39FEC9E4049
:1024D9000F9007BFE0F8A3E09007B9C8F0A3C8F0D0
:1024E900229006C8E090386BF8282873804C8553F1
:1024F9007380479000D4E0855FF0A4FFAEF07408C4
:102509001200398F738033856173802E85677380DC
:10251900298568738024856973801F856A73801A89
:10252900856B7380158566738010856573800B854F
:0A2539006C73800690001AE0F57341
:10386B000224F50224F70224FC022510022515027E
:10387B00251A02251F02252402252902252E0225A1
:07388B003302253802253D40
:102543009006C9E0FE9006CAE0D39E404B9006C8B1
:10255300E0B404189006CAE0C395735002D22D90DC
:1025630006C9E0D395734002C22D802A9006C9E0C4
:10257300C3957350099006CAE0D395735002800245
:10258300D22D9006C9E0D3957350099006CAE0C3D3
:1025930095735002C22D802A9006C9E0D3957340EB
:1025A300099006CAE0C3957340028002C22D9006CB
:1025B300C9E0C3957340099006CAE0D395734002FE
:1025C300D22D229006CCE0903892F8282873804CC4
:1025D30085537380479000D4E0855FF0A4FFAEF08D
:1025E30074081200398F738033856173802E856779
:1025F3007380298568738024856973801F856A7356
:10260300801A856B7380158566738010856573806A
:0C2613000B856C73800690001AE0F573D4
:103892000225D10225D30225D80225EC0225F10208
:1038A20025F60225FB02260002260502260A02262A
:0738B2000F02261402261983
:10261F009006CDE0FE9006CEE0D39E405F9006CCB4
:10262F00E0B404189006CEE0C395735002D22E90FA
:10263F0006CDE0D395734002C22E803E9006CDE0CA
:10264F00C3957350099006CEE0D395735002800264
:10265F00D22E9006CDE0D3957350099006CEE0C3ED
:10266F0095735002C22E9006CCE0B401099000E0A1
:10267F00E0D3956150028002C22E802A9006CDE0F1
:10268F00D3957340099006CEE0C395734002800244
:10269F00C22E9006CDE0C3957340099006CEE0D3CD
:1026AF0095734002D22E229006D0E09038B9F828C8
:1026BF002873804C85537380479000D4E0855FF07A
:1026CF00A4FFAEF074081200398F738033856173E5
:1026DF00802E856773802985687380248569738050
:1026EF001F856A73801A856B7380158566738010DA
:1026FF00856573800B856C73800690001AE0F57307
:1038B9000226C10226C30226C80226DC0226E1022C
:1038C90026E60226EB0226F00226F50226FA022651
:0738D900FF0227040227098A
:10270F009006D1E0FE9006D2E0D39E404B9006D0CB
:10271F00E0B404189006D2E0C395735002D22F9004
:10272F0006D1E0D395734002C22F802A9006D1E0E4
:10273F00C3957350099006D2E0D39573500280026F
:10274F00D22F9006D1E0D3957350099006D2E0C3F3
:10275F0095735002C22F802A9006D1E0D395734013
:10276F00099006D2E0C3957340028002C22F9006F3
:10277F00D1E0C3957340099006D2E0D39573400220
:10278F00D22F229006D4E09038E0F8282873804C9E
:10279F0085537380479000D4E0855FF0A4FFAEF0BF
:1027AF0074081200398F738033856173802E8567AB
:1027BF007380298568738024856973801F856A7388
:1027CF00801A856B7380158566738010856573809D
:0C27DF000B856C73800690001AE0F57307
:1038E00002279D02279F0227A40227B80227BD02B4
:1038F00027C20227C70227CC0227D10227D60227D8
:07390000DB0227E00227E5CE
:1027EB009006D5E0FE9006D6E0D39E404B9006D4E3
:1027FB00E0B404189006D6E0C395735002D2309023
:10280B0006D5E0D395734002C230802A9006D5E0FE
:10281B00C3957350099006D6E0D39573500280028E
:10282B00D2309006D5E0D3957350099006D6E0C30D
:10283B0095735002C230802A9006D5E0D395734031
:10284B00099006D6E0C3957340028002C230900611
:10285B00D5E0C3957340099006D6E0D3957340023B
:10286B00D230229006D8E0903907F8282873804C94
:10287B0085537380479000D4E0855FF0A4FFAEF0E2
:10288B0074081200398F738033856173802E8567CE
:10289B007380298568738024856973801F856A73AB
:1028AB00801A856B738015856673801085657380C0
:0C28BB000B856C73800690001AE0F5732A
:1039070002287902287B022880022894022899023B
:10391700289E0228A30228A80228AD0228B202285E
:07392700B70228BC0228C111
:1028C7009006D9E0FE9006DAE0D39E404B9006D8FA
:1028D700E0B404189006DAE0C395735002D2319041
:1028E70006D9E0D395734002C231802A9006D9E019
:1028F700C3957350099006DAE0D3957350028002AE
:10290700D2319006D9E0D3957350099006DAE0C327
:1029170095735002C231802A9006D9E0D39573404F
:10292700099006DAE0C3957340028002C23190062F
:10293700D9E0C3957340099006DAE0D39573400256
:10294700D231229006DCE090392EF8282873804C8B
:1029570085537380479000D4E0855FF0A4FFAEF005
:1029670074081200398F738033856173802E8567F1
:102977007380298568738024856973801F856A73CE
:10298700801A856B738015856673801085657380E3
:0C2997000B856C73800690001AE0F5734D
:10392E0002295502295702295C02297002297502C3
:10393E00297A02297F02298402298902298E0229E5
:07394E009302299802299D54
:1029A3009006DDE0FE9006DEE0D39E404B9006DC11
:1029B300E0B404189006DEE0C395735002D232905F
:1029C30006DDE0D395734002C232802A9006DDE033
:1029D300C3957350099006DEE0D3957350028002CD
:1029E300D2329006DDE0D3957350099006DEE0C342
:1029F30095735002C232802A9006DDE0D39573406E
:102A0300099006DEE0C3957340028002C23290064D
:102A1300DDE0C3957340099006DEE0D39573400271
:102A2300D232229006E0E0903955F8282873804C82
:102A330085537380479000D4E0855FF0A4FFAEF028
:102A430074081200398F738033856173802E856714
:102A53007380298568738024856973801F856A73F1
:102A6300801A856B73801585667380108565738006
:0C2A73000B856C73800690001AE0F57370
:10395500022A31022A33022A38022A4C022A51024B
:103965002A56022A5B022A60022A65022A6A022A6C
:073975006F022A74022A7997
:102A7F009006E1E0FE9006E2E0D39E404B9006E028
:102A8F00E0B404189006E2E0C395735002D233907D
:102A9F0006E1E0D395734002C233802A9006E1E04D
:102AAF00C3957350099006E2E0D3957350028002EC
:102ABF00D2339006E1E0D3957350099006E2E0C35C
:102ACF0095735002C233802A9006E1E0D39573408C
:102ADF00099006E2E0C3957340028002C23390066C
:102AEF00E1E0C3957340099006E2E0D3957340028D
:102AFF00D233229006E4E090397CF8282873804C7A
:102B0F0085537380479000D4E0855FF0A4FFAEF04B
:102B1F0074081200398F738033856173802E856737
:102B2F007380298568738024856973801F856A7314
:102B3F00801A856B73801585667380108565738029
:0C2B4F000B856C73800690001AE0F57393
:10397C00022B0D022B0F022B14022B28022B2D02D3
:10398C002B32022B37022B3C022B41022B46022BF3
:07399C004B022B50022B55DA
:102B5B009006E5E0FE9006E6E0D39E404B9006E43F
:102B6B00E0B404189006E6E0C395735002D234909B
:102B7B0006E5E0D395734002C234802A9006E5E067
:102B8B00C3957350099006E6E0D39573500280020B
:102B9B00D2349006E5E0D3957350099006E6E0C376
:102BAB0095735002C234802A9006E5E0D3957340AA
:102BBB00099006E6E0C3957340028002C23490068A
:102BCB00E5E0C3957340099006E6E0D395734002A8
:102BDB00D234229006E8E09039A3F8282873804C71
:102BEB0085537380479000D4E0855FF0A4FFAEF06F
:102BFB0074081200398F738033856173802E85675B
:102C0B007380298568738024856973801F856A7337
:102C1B00801A856B7380158566738010856573804C
:0C2C2B000B856C73800690001AE0F573B6
:1039A300022BE9022BEB022BF0022C04022C09025E
:1039B3002C0E022C13022C18022C1D022C22022C7A
:0739C30027022C2C022C311D
:102C37009006E9E0FE9006EAE0D39E404B9006E856
:102C4700E0B404189006EAE0C395735002D23590B9
:102C570006E9E0D395734002C235802A9006E9E081
:102C6700C3957350099006EAE0D39573500280022A
:102C7700D2359006E9E0D3957350099006EAE0C390
:102C870095735002C235802A9006E9E0D3957340C8
:102C9700099006EAE0C3957340028002C2359006A8
:102CA700E9E0C3957340099006EAE0D395734002C3
:102CB700D235229006ECE09039CAF8282873804C68
:102CC70085537380479000D4E0855FF0A4FFAEF092
:102CD70074081200398F738033856173802E85677E
:102CE7007380298568738024856973801F856A735B
:102CF700801A856B73801585667380108565738070
:0C2D07000B856C73800690001AE0F573D9
:1039CA00022CC5022CC7022CCC022CE0022CE502E8
:1039DA002CEA022CEF022CF4022CF9022CFE022D06
:0739EA0003022D08022D0D60
:102D13009006EDE0FE9006EEE0D39E404B9006EC6D
:102D2300E0B404189006EEE0C395735002D23690D7
:102D330006EDE0D395734002C236802A9006EDE09B
:102D4300C3957350099006EEE0D395735002800249
:102D5300D2369006EDE0D3957350099006EEE0C3AA
:102D630095735002C236802A9006EDE0D3957340E6
:102D7300099006EEE0C3957340028002C2369006C6
:102D8300EDE0C3957340099006EEE0D395734002DE
:102D9300D23622AE2EAF2F74F5D39F74019E400816
:102DA300782E126B03022EB0752F01752E00AE52D2
:102DB300AF53E546BE000DD39F40099000B6E0D364
:102DC300954740028023754700E546C39553F57345
:102DD3009000B9E0D395454008E5452573F5458056
:102DE300069000B9E0F54580020547900092E0D3D4
:102DF3009561401CE55FC395604015AE52AF53E546
:102E030046BE00039F50099000B7E0D395484002A7
:102E1300806E9007D2E0A852B80004955350037512
:102E23004A009007D2E0A852B8000BD3955340064E
:102E3300E5539007D2F0E54A7041E553C39546F553
:102E430073E573D3940540037573059000B8E0C32D
:102E530095455007E573C3954540028009E545C391
:102E63009573F54580069000B8E0F5459000B8E00D
:102E7300D3954540069000B8E0F5457548008002BB
:102E83000548E54A7016900092E0C39561500DE540
:102E9300462405A852B8000695534002800F9000BF
:102EA300A5E0F545754A0174789007D2F022AE2E5D
:102EB300AF2F74E9D39F74039E4008782E126B03DF
:102EC30002304F752F01752E00754532A237402A07
:102ED3007545199000A5E075F002A4FFAEF0E54733
:102EE300BE0006D39F4002D2370547754A03747864
:102EF3009007D2F075490002303EAE52AF53E5461B
:102F03006F4E700302303EE546BE000DD39F40096D
:102F13009000B6E0D395474002800F754700E54A1D
:102F2300C394035003754519800DE546C39553F5C6
:102F330073E5472573F547900092E0D39561400E02
:102F43009007D2E0A852B80007D395534002800CF3
:102F530005499000A5E0B54903754A00E54AB40365
:102F630006A20DB3B34002800A0549E549B43C0308
:102F7300754A02E54AB402299007D2E0A852B80084
:102F83000ED395534009E5539007D2F0754900904D
:102F93000092E0C39561500975490074789007D297
:102FA300F0E54A705A900092E0D39561401CE55FCA
:102FB300C395604015AE52AF53E546BE00039F5024
:102FC300099000B7E0D39548400280087548007522
:102FD300454B8028E553C39546F573E573D39405B4
:102FE3004003757305900092E0D395614008E5486E
:102FF3002573F5488006E5482406F548754900E53C
:103003004A7016900092E0C39561500DE546240581
:10301300A852B80006955340028003754A01E54A59
:10302300B4011875451905499000A5E0B549067521
:103033004A0275490074789007D2F0E54575F00AA5
:10304300A4FFAEF09007C3EEF0A3EFF022E56F907C
:1030530039F1F828287390008AE0700302327790E0
:1030630000C0E0B40102800302319290004DE0B54C
:103073005E02800302318F7E017F00E5BE126AAFDC
:10308300E5BD2FFF50010E8E5A8F5B7410126AAF8D
:10309300900078E08E048F05FF126A9F9007C7ECBB
:1030A300F0A3EDF074FFBC00039D500B74FF900779
:1030B300C7F8E4F0E8A3F0E56B600FE56BC394FE9B
:1030C30050089000E6E06402600280649000D4E05F
:1030D300B40B1F9007C7E0FEA3E0FF74E7126AAFCB
:1030E300E56B8E048F05FF126A9F9007C7ECF0A370
:1030F300EDF09000D4E0D3940B40089000BCE06462
:10310300046002802B9007C7E0FEA3E0FF9007C98D
:10311300E0FCA3E0FDEFD39DEE9C400D126AFB9013
:1031230007C7EEF0A3EFF080079007C7E4F0A3F022
:1031330090008AE0B4021E9007C7E0FEA3E0FF9070
:1031430007D3E02FFF50010E74011200399007C717
:10315300EEF0A3EFF09007C7E0FEA3E0FF9007D3E4
:10316300E0BE0008D39F4004D23A8002B23A9007EF
:10317300C8E09007D3F09000BCE064016006A23A77
:10318300B3B3400280069007C8E0F55F023275D200
:103193003A7E017F00E5BE126AAFE5BD2FFF500105
:1031A3000E8E5A8F5B7410126AAF900078E08E0413
:1031B3008F05FF126A9F9007C7ECF0A3EDF0E56B54
:1031C300600FE56BC394FE50089000E6E064026074
:1031D3000280649000D4E0B40B1F9007C7E0FEA305
:1031E300E0FF74E7126AAFE56B8E048F05FF126A86
:1031F3009F9007C7ECF0A3EDF09000D4E0D3940BBD
:1032030040089000BCE064046002802B9007C7E094
:10321300FEA3E0FF9007C9E0FCA3E0FDEFD39DEE22
:103223009C400D126AFB9007C7EEF0A3EFF08007F6
:103233009007C7E4F0A3F090008AE0B4021E900761
:10324300C7E0FEA3E0FF9007D3E02FFF50010E7409
:10325300011200399007C7EEF0A3EFF09007C8E022
:103263009007D3F09000BCE0640160069007C8E0CB
:10327300F55F8003755F00900086E07006756F014F
:1032830002305075BB18023845900086E070030287
:1032930033FD7E017F00E5BE126AAFE5BD2FFF500F
:1032A300010E8E5A8F5B9000CCE0B4010F7E0F7F2E
:1032B300FFAC5AAD5B126AFB8E5A8F5B9000F1E054
:1032C300B40245AE5AAF5B900023E0FCA3E0FDEDF2
:1032D300D39FEC9E400A900023E55AF0A3E55BF0F0
:1032E300AE5AAF5B900025E0FCA3E0FDEFD39DEE6B
:1032F3009C400A900025E55AF0A3E55BF0AE5AAF77
:103303005B74041200398F619000F1E0704CAE5A87
:10331300AF5B900023E0FCA3E0FDEFD39DEE9C4068
:1033230009126AFB8E5A8F5B8006755B00755A0023
:10333300AE5AAF5B7410126AAF900075E08E048FC3
:1033430005FF126A9F8C5A8D5B74FFBC0009D39DE5
:103353004005855B6180037561FE9000BCE0B401AC
:103363000280030233FBA20DB3B3500E900090E032
:10337300A852B80005D39553500280719000CDE058
:103383008561F0A4FFAEF074648E048F05FF126AAA
:103393009F8C5A8D5BE56B6016E56BC394FE500FF3
:1033A3009000E6E0B402089000D4E0640B60028071
:1033B30017AE5AAF5B74E7126AAFE56B8E048F05E5
:1033C300FF126A9F8C5A8D5BAE5AAF5B9007C7E0C2
:1033D300FCA3E0FDEDD39FEC9E4005855B5F800B76
:1033E300A23AB340069007C8E0F55F800BA23AB358
:1033F30040069007C8E0F55F80037561009000897F
:10340300E07006756F0202305075BB1902384590A3
:103413000089E070030234B2E55ED39551400302A4
:1034230034B0900021E0FEA3E0FFE565126AF3905B
:103433000021EEF0A3EFF07E017F00E5BE126AAF3C
:10344300E5BD2FFF50010E8E5A8F5B9000F6E070A2
:1034530013740A126AAF74518E048F05FF126A9FA8
:103463008D658019AE5AAF5B740A126AAF8F048EF2
:10347300057E017F95CDCCCD12699D8F65E565D322
:1034830094644003756564900021E0FEA3E0FFE5CA
:10349300652FFF50010E900021EEF0A3EFF0900096
:1034A3008DE0048E048F05FF126A9F8D658003757E
:1034B30065329000D9E07006756F0302305075BB1A
:1034C300130238459000D9E0604A7E017F00E5BED3
:1034D300126AAFE5BD2FFF50010E8E5A8F5B740445
:1034E3001200398F669000DBE08566F0A4FDACF036
:1034F3007464FF126A9F8D669000DAE08566F0A41B
:10350300FFAEF074FF8E048F05FF126A9FED9000EB
:1035130074F08003756600900087E07006756F0491
:1035230002305075BB17023845900087E0B40102A2
:1035330080030235C07E017F00E5BE126AAFE5BDA0
:103543002FFF50010E8E5A8F5B9007D4E0601990C5
:1035530007D4E01490640F12008CE493FC7401937D
:10356300FDEDC39FEC9E400280069007D4E014F06B
:103573009007D4E0C394B3501DAE5AAF5B9007D409
:10358300E00490640F12008CE493FC740193FDEF4C
:10359300C39DEE9C400280069007D4E004F09007A0
:1035A300D4E0FE9000ADE08E0088F0A4FFAEF0748E
:1035B300648E048F05FF126A9F8D67800375670011
:1035C300900088E07006756F0502305075BB1602D7
:1035D3003845900088E0B4010280030236697E0119
:1035E3007F00E5BE126AAFE5BD2FFF50010E8E5A74
:1035F3008F5B9007D5E060199007D5E0149065794B
:1036030012008CE493FC740193FDEDC39FEC9E4088
:103613000280069007D5E014F09007D5E0C394B379
:10362300501DAE5AAF5B9007D5E004906579120048
:103633008CE493FC740193FDEFC39DEE9C400280E8
:10364300069007D5E004F09007D5E0FE9000B3E0C4
:103653008E0088F0A4FFAEF074648E048F05FF1211
:103663006A9F8D68800375680075BB1F0238457EAD
:10367300017F00E5BE126AAFE5BD2FFF50010E8E3C
:103683005A8F5B7409126AAF74E68E048F05FF12BA
:103693006A9F8D6A90008FE07006756F0702305045
:1036A30075BB1502384590008FE070030237C47E66
:1036B300017F00E5BE126AAFE5BD2FFF50010E8EFC
:1036C3005A8F5B74041200398F6990008FE0B40144
:1036D300159000E3E08569F0A4FFAEF074071200D3
:1036E30039EF9007CCF090008FE0B402159000E31F
:1036F300E08569F0A4FFAEF07407120039EF90077C
:10370300CBF090008FE0B4030280030237A7900050
:10371300D0E0701CE569C394195002D22CE569D33B
:1037230094644002C22C9000AFE09007CFF0806316
:103733009000AFE070349000E3E08569F0A4FFAE41
:10374300F074FF8E048F05FF126A9FED9007CFF090
:10375300AE52AF53741EBE0006D39F4002D22CE577
:1037630061D394E54002C22C8029E569C3940A50D1
:103773000DAE52AF53741EBE0004D39F500280029D
:10378300D22CE561D394E54002C22C9000AFE090C7
:1037930007CFF09007CFE0C3940550067405900758
:1037A300CFF0C23B90008FE0B40414E569C39419D1
:1037B3005002D23BE569D394324002C23BC22C8013
:1037C300037569009000E6E07006756F08023050DB
:1037D30075BB14806D9000E6E060567E017F00E5C6
:1037E300BE126AAFE5BD2FFF50010E8E5A8F5BEFFD
:1037F300D39421EE940E4005756BFF8015AE5AAF3E
:103803005B7410126AAF74E38E048F05FF126A9F14
:103813008D6BE56B75F00BA4FFAEF09000D4E08EDA
:10382300048F05FF126A9F9007C9ECF0A3EDF080A7
:1038330003756B0090008AE0600575BB1A80037501
:02384300BB18B0
:1039F10002305902328C0234120234C702352C02D1
:0B3A010035D50236720236A90237D814
:05384500056FD2EC222A
:096AE1002582F582500205832292
:0F008C0025E050020583258250020583F582226C
:106A7E00EF2F500205832582F582E5833E2EF583A6
:016A8E0022E5
:106AF300CFC39FFF50011E22C3EF9DFFEE9CFE22DA
:086B03000806B6000218062284
:0D6ABD00A3E004F07006120049E004F0228E
:0E003900048007C3CE13CECF13CFD5E0F6223E
:10699D00BC000FBE0008ED8FF084FFADF022E4FEC9
:1069AD00FF22BE000DEF60FE54F0606F20E7030282
:1069BD006A53EAC0E0EBC0E078017A0075F001EEB1
:1069CD0020E710EF25E0FFEE33FE0AC5F023C5F0FA
:1069DD0030E7F0EA5407F9096A7A007B0060010894
:1069ED00C3EC9E40167004ED9F4010ED9FFDEC9E94
:1069FD00FCE5F0CA4ACA03F5F08005E5F003F5F0B1
:106A0D00C3EE13FEEF13FFD9D77908CACBCAD8D07E
:106A1D00EAFEEBFFD0E0FBD0E0FA22EC8FF084FC35
:106A2D00ED54F045F0C48FF084FEEDC454F045F004
:106A3D00C48FF084FDEEC4FE54F02DFFEE540F3CD8
:106A4D00FEADF07C0022790078008FF0EC7E0820FE
:106A5D00E70DC3CD33CD33C933C9C833C8DEF08498
:106A6D0049F9E5F08FF0BE00E6FD7C00E9FFE8FE98
:016A7D0022F6
:0E6AAF00F88FF0A4FFE5F0CE88F0A42EFE22B2
:10000300EF8DF0A4F9A8F0EF8CF0A428F8EE8DF0B2
:06001300A428FEE9FF2213
:106A8F00600D782B026A99007830D8FED5E0F82295
:106A9F00EEC0E07E0012699DEFFDEEFCD0E0FE221D
:0C6ACA00EEC0E07E0012699DD0E0FE22CC
:03001B0002001EC2
:0300530002005652
:03009B00020071EF
:03000000026AEAA7
:096AEA0075817575D0000244733A
:0B6AD600E5822FF582E5833EF5832268
:0A0049000582D5820215831582227C
:10001E00C0E0C0F0C083C082C0D075D0001243DFF4
:0B002E00D0D0D082D083D0F0D0E032E0
:10005600C0E0C0F0C083C082C0D075D0001243E2B9
:10006600D0D0D082D083D0F0D0E032C0E0C0F0C093
:1000760083C082C0D075D0001243FED0D0D082D0CB
:0600860083D0F0D0E0324F
:00000001FF
